:020000040000fa
:20000000001000207f01000075010000770100000000000000000000000000000000000042
:020000040000fa
:200020000000000000000000000000007501000075010000000000007501000075010000e8
:020000040000fa
:2000400075010000750100007501000075010000750100007501000075010000ed04000075
:020000040000fa
:200060007501000075010000750100007501000075010000750100007501000075010000d0
:020000040000fa
:200080007501000075010000750100007501000075010000750100007501000075010000b0
:020000040000fa
:2000a0007501000075010000750100007501000075010000750100000000fdff020012016b
:020000040000fa
:2000c000100102000020feff0a0000010102030109024300020100c0320904000001020289
:020000040000fa
:2000e000010005240010010524010101042402020524060001070581030800ff0904010098
:020000040000fa
:20010000020a000000070504024000000705850240000004030904200361006c00740075c1
:020000040000fa
:200120000073006d0065007400720075006d002e006f0072006700160341006c0074006f93
:020000040000fa
:2001400000730046006c006100730068000e0330003000300030003000310000000000000c
:020000040000fa
:2001600010b500f0b9f800f0f1fc00f0b9fd002010bd000070470e2010b500f0a8fd10b5a5
:020000040000fa
:200180000f49104a104800f043fe00210f4a104800f047fe00f040f8002807d000f06cf8a2
:020000040000fa
:2001a000002803d08020400100f026f80423094a91690b439361084b084a9360fff7d0ff42
:020000040000fa
:2001c000c60e0000300000000c000020740200003c000020000400400000000000ed00e00c
:020000040000fa
:2001e000044b98689b6880b25b035b0f033398407047c046004000414368064a591eff39bd
:020000040000fa
:20020000914205d8da0703d5026895469e4670477047c04600ff1f000a4b0b4a596810b58a
:020000040000fa
:20022000914203d1094a9968914201d0012010bd00225a609a601b6818009342f7d0fff72e
:020000040000fa
:20024000dbfff3e700000020a5a55a5a3c3cc3c3044b054a18605a60044a9a60044b054a18
:020000040000fa
:20026000da60704700000020a5a55a5a3c3cc3c300ed00e00400fa050823114a10b5d1691c
:020000040000fa
:2002800010480b43d3618023db024360836147230d490c789c43413b23430b706423c04670
:020000040000fa
:2002a000013b9bb2002bfad10424006a0b784003a3430b700821d369c00f8b43d36110bd03
:020000040000fa
:2002c00000040040004400415244004130bf62b672b60020704770470223284830b542689d
:020000040000fa
:2002e0000124134343600c2325498a691343254a8b6114701378234203d053785bb2002b55
:020000040000fa
:20030000f8db214b214c1c6102241d692c431c610124dd682542fcd01d4cdc641d4c9c646d
:020000040000fa
:2003200000245c645d6c02342c435c6404241d6d2542fcd002241d6d2542fcd0547864b201
:020000040000fa
:20034000002cfbdb00249460547864b2002cfbdb842464025460547864b2002cfbdb0022d7
:020000040000fa
:200360000a724a728a72ca7202211a6a8a431a62802342681343436030bdc0460040004163
:020000040000fa
:2003800000040040000c00400008004044d3000014007f00ff020000044b1a78012a03d8f3
:020000040000fa
:2003a000511c1970013398547047c0463c00002070b50d4b0d4d5b68ea789b049b0c1c1c94
:020000040000fa
:2003c000934200d9141c29006e68a4b2121bea7030002200083100f01bfd4022044b3619d0
:020000040000fa
:2003e0006e605a7170bdc046b00100203c000020ff500041f8b5124ef3795bb2002b1edbca
:020000040000fa
:20040000104d20242b781f2b04d82a0000211c00283211702800ef6a1b1b220039003030be
:020000040000fa
:200420002b7000f0f5fc084a3f195369ef621b0f1b071c4380235461b371783b3372f8bd55
:020000040000fa
:20044000ff5000413c000020b001002010b501240548064a037812781341234200d110bdfc
:020000040000fa
:20046000fff734fff4e7c0468c0000208d000020012030b5194a1a4b117802001c008a40da
:020000040000fa
:20048000503425782a4322701a0052321478402c02d01a00533210700800124a0a30000116
:020000040000fa
:2004a00012185068a625000f00070443546001221400881d8440e0b20b4cff3560551500f7
:020000040000fa
:2004c000881c8540e8b2a825ff3560551800521a51300270002252331a7030bd8d00002021
:020000040000fa
:2004e0003c000020b0010020005000410120f0b5c74d85b0ab8b9bb202932b8c9ab203927f
:020000040000fa
:20050000029aaa8303427cd0c24ac349137a0226dbb21372c14c0a78df0600d4bde0024378
:020000040000fa
:200520000a70334205d022000423543211780b431370230054331a78019200221a7001232f
:020000040000fa
:20054000019f019a1f401a4230d0260007335636e3706660fff72cffe378002b26d10022e0
:020000040000fa
:20056000b2563378002a03dbf288002a00d00227220028321770621ce26200221800227092
:020000040000fa
:2005800060321040134200d18ce0202800d16be1a34aa24b1278012a08d11a005632d2881e
:020000040000fa
:2005a0001978914200d91a70fff724ff019b9b0711d59b4e994c3378022b0cd1fff7f8fec8
:020000040000fa
:2005c000e378002b07d1012232702278002a00d02370fff70fff019b5b0712d5904b8f4c32
:020000040000fa
:2005e0001b78012b01d1fff705ff22005f321378002b06d080215e3423780b43ab720023d5
:020000040000fa
:200600001370039bdb0612d58822ff32ab5c0321dbb2ab541a000a400b4208d08148037892
:020000040000fa
:20062000134301220370804b1a70fff754fe039b9b0610d5a822ff32ab5cdbb21900ab5466
:020000040000fa
:20064000a53aff3a1140134205d0784803788b430370fff740fe029b1b071cd56f4b744a2f
:020000040000fa
:200660007449180011608021303089055160106151611121674a5170ee315171ec39917224
:020000040000fa
:20068000190000226e310a70190028310a70da621a705a60da7005b0f0bd034200d140e7b1
:020000040000fa
:2006a00032433de71f221340012b00d1a8e0022b00d1cde0002b00d06ae723005633587815
:020000040000fa
:2006c000092800d964e700f099fbc80063ff63ff63ff63ff0a00140063ff340037002200e4
:020000040000fa
:2006e0002300563252885e331a7001235f3423704ee72300563359884f4a0e0af7b2c9b279
:020000040000fa
:200700001378002b00d143e75078b8420fd1481ec0b200290ad1022e00d1937821005631f6
:020000040000fa
:20072000c988994200d2cbb2e262e0e70100d218e6e76034207894e0230056335b883f4ac3
:020000040000fa
:200740000026137022003a4b64321e625e621a6390224021ff2752005e63a9540432af5474
:020000040000fa
:200760002a220221ff32a954354a191dca671900c022180092050831ca6732499030016046
:020000040000fa
:20078000190094310a60c02153204900685404316f548a2103205f3fbc46ff316854210045
:020000040000fa
:2007a0009c44674602386c31087027493960b027bc4619009c446746a4310a602349b43343
:020000040000fa
:2007c00039601a60d0233522ff275b00ea540433ef54aa230322ff33ea54230051331e70ec
:020000040000fa
:2007e000230053331870200050300670fff773fd2000124b6d3006701e70fff76cfdc7e622
:020000040000fa
:2008000056346378002b28d00a2b00d0c0e628e000500041ff500041900000203c00002070
:020000040000fa
:2008200064000020a9000020aa0000208c000020b001002044000020be0000009c00002046
:020000040000fa
:20084000b0000020f0000020300100207001002056346378002b00d09ae60020fff79cfd47
:020000040000fa
:200860000020fff799fd93e6230056335b78202b06d0212b00d08be6044be362072336e74b
:020000040000fa
:20088000024b63600723e37082e6c0460c00002010b5094b094c1b78002b0cd072b653347a
:020000040000fa
:2008a0002378002b06d1fff7d1fd2378002b01d1fff7defd62b610bdaa0000203c00002063
:020000040000fa
:2008c00070b5114b05001b78104c002b1bd072b6fff7bcfd2300002253331a7023005234b8
:020000040000fa
:2008e0005133207819780a4b421c8901d2b25b1822701d54402a01d1fff7bafd62b60a2ddc
:020000040000fa
:2009000001d1fff7c5ff70bdaa0000203c00002030010020f8b572b601242f4b2f481b7829
:020000040000fa
:20092000002b32d002006c321778020003006d321178002270331d78030094466f331b78c2
:020000040000fa
:20094000274eab4225d10d00e21bd2b2154125420cd0230093409943130008331b01f318d1
:020000040000fa
:200960005b681700a4460025dbb2eae76246002a0bd002006c32177002006d321170020038
:020000040000fa
:200980006f3213700200703213706d30fff79efcc3e76246002a08d002006c321770020062
:020000040000fa
:2009a0006d32117002006f32137002006c3211786c1c70300b4ae4b2047088011218505de1
:020000040000fa
:2009c000a34207d1012306318b40c2220649dbb252008b5462b6f8bdaa0000203c00002050
:020000040000fa
:2009e000b0010020b00000200050004172b68022084bda67084b7f3a19890a4302211a81ae
:020000040000fa
:200a00001a788a431a70054a1e31d3698b43d36162b6704704e100e00050004100040040a8
:020000040000fa
:200a2000f8b508233e490f25ca693e481343cb61062302783c4caa43134303700123227849
:020000040000fa
:200a40009a431a432270602204782c4022430270364802789a4313430370354a354b538019
:020000040000fa
:200a600053785bb2002bfbdb2023ca69324c13430122cb6123781343237023781342fcd1c3
:020000040000fa
:200a80000125a378190029402b42fad180222b4e5200300000f0c5f92389294a1d432581eb
:020000040000fa
:200aa0006662106a516a8b03db0e1f2b00d11a3b106a516a4902c90e1f2900d10239166a27
:020000040000fa
:200ac000576aba01520f072a00d1043a9b010b431203134323850f23e37072b60023238188
:020000040000fa
:200ae00006332370043ba2781a42fcd18023c1208021144a80001360135889041b021b0af8
:020000040000fa
:200b00000b4313500823238362b60f4bc046013b002bfbd10122238993432381f8bdc046a4
:020000040000fa
:200b2000000400403c4400415844004159440041000c00400640000000500041b001002001
:020000040000fa
:200b40000060800000e100e050c3000010b5fff767ff0022014b1a7010bdc0466400002071
:020000040000fa
:200b60000122054b59691142fcd001224008d86159691142fcd0704700400041f7b504268e
:020000040000fa
:200b8000194f0400bb685b035b0f03339e40731e184224d172b63500ff352d0a013d3b6a5f
:020000040000fa
:200ba0000193fff71dfb23000009002818d1ff221340019ada4013000122134205d02000ad
:020000040000fa
:200bc000fff7ceff412000f037f92000fff7c8ff022000f031f9a419013de0d262b6f7bd3f
:020000040000fa
:200be0005b084008e1e7c04600400041f7b58026154b76009c6805006403640fe31c1e4192
:020000040000fa
:200c000001230134a3400f000193fff7b7ff72b60423a3401c00002e01d162b6f7bd4420cb
:020000040000fa
:200c200000f00af92800fff79bff00239a00b9580133a950019a9a42f8d1042000f0fcf8c6
:020000040000fa
:200c40003f192d19013ee6e70040004170b5040045182678002e0ad00a2e02d10d20fff70f
:020000040000fa
:200c60002ffe30000134fff72bfeac42f1d170bd70b505001c240f262800e04030400a285d
:020000040000fa
:200c800000d927303030043cfff71afe231df3d170bd10b5fff73efe2028fbd00024030014
:020000040000fa
:200ca000303b092b05d8180024010443fff732fef5e70300613b052b01d85738f4e703001d
:020000040000fa
:200cc000413b052b01d83738eee7200010bdfee710b50249fff7baff10bdc046ffff0000e9
:020000040000fa
:200ce000f0b580248025c1b064016d00fff7d0fdfff710fe58284bd01bd852284dd0572858
:020000040000fa
:200d0000f4d1fff7c6ff00270600fff703fe6b46d8550137af42f8d1a642e7d3fff760fa6d
:020000040000fa
:200d20000138ff388642e1d869463000fff75effdce7612828d07628d8d12748fff7c8ffd9
:020000040000fa
:200d40002648fff7c5ff2648fff7c2ff2548fff7bfff2548fff7bcff2448fff7b9ff2000cd
:020000040000fa
:200d6000fff786ff2020fff7abfdfff739fafff77fff1f48fff7acff08211e48fff766ff8b
:020000040000fa
:200d80001d48fff7a5ffb1e72000fff761faade7fff77ffffff7f2fea8e7fff77aff060059
:020000040000fa
:200da000a04208d22e00013eff20b6b2fff788fd002ef8d19ae7fff713fa0138ff38864255
:020000040000fa
:200dc000f0d8771cff37330001361878fff778fdbe42f8d18ae7c0466b0e0000780e0000de
:020000040000fa
:200de000530e00008b0e0000480e00009e0e0000b10e0000630e0000c40e000003b4714687
:020000040000fa
:200e0000490840004900095e49008e4403bc7047002310b59a4200d110bdcc5cc45401332a
:020000040000fa
:200e2000f8e703008218934200d1704719700133f9e700000000000001b40248844601bcb6
:020000040000fa
:200e4000604700bf19000020416c746f73466c61736800616c7475736d657472756d2e6fa2
:020000040000fa
:200e6000726700312e392e31370000616c746f732d6c6f61646572000a6d616e75666163bf
:020000040000fa
:200e800074757265722020202020000a70726f6475637420202020202020202020000a66c5
:020000040000fa
:200ea0006c6173682d72616e6765202020202020000a736f6674776172652d7665727369c5
:020000040000fa
:200ec0006f6e20000a0000c2010000000800000000000122074b59691142fcd0a52212020f
:020000040000fa
:200ee00010430122186059691142fcd003225a617047004000410000ffffffffffffffff13
:020000040000fa
:200f0000fffffffffffffffffffffffffffffffffffffffffffffffffffffffffffffffff1
:020000040000fa
:200f2000ffffffffffffffffffffffffffffffffffffffffffffffffffffffffffffffffd1
:020000040000fa
:200f4000ffffffffffffffffffffffffffffffffffffffffffffffffffffffffffffffffb1
:020000040000fa
:200f6000ffffffffffffffffffffffffffffffffffffffffffffffffffffffffffffffff91
:020000040000fa
:200f8000ffffffffffffffffffffffffffffffffffffffffffffffffffffffffffffffff71
:020000040000fa
:200fa000ffffffffffffffffffffffffffffffffffffffffffffffffffffffffffffffff51
:020000040000fa
:200fc000ffffffffffffffffffffffffffffffffffffffffffffffffffffffffffffffff31
:020000040000fa
:200fe000ffffffffffffffffffffffffffffffffffffffffffffffffffffffffffffffff11
:020000040000fa
:20100000004000203f1200003512000037120000000000000000000000000000000000008f
:020000040000fa
:2010200000000000000000000000000035120000351200000000000035120000e1250000d5
:020000040000fa
:20104000351200003512000035120000351200002544000035120000d92700005d3e000029
:020000040000fa
:20106000351200003512000035120000351200003512000035120000351200003512000038
:020000040000fa
:201080003512000035120000351200003512000035120000351200003512000059390000cd
:020000040000fa
:2010a0003512000035120000351200003512000035120000351200000000fdff0200120175
:020000040000fa
:2010c000100102000020feff0d0000010102030109024300020100c0320904000001020276
:020000040000fa
:2010e000010005240010010524010101042402020524060001070581030800ff0904010088
:020000040000fa
:20110000020a000000070504024000000705850240000004030904200361006c00740075b1
:020000040000fa
:201120000073006d0065007400720075006d002e006f00720067001a03450061007300797d
:020000040000fa
:2011400000540069006d00650072002d00760032000e033000300030003000300031000087
:020000040000fa
:2011600010b501f091fa00f081fe01f077fa01f0cbfb01f09dfe03f00ffa02f04bfc02f0f3
:020000040000fa
:20118000f1fc00f0f5fa01f09ff902f01ff802f0c3f904f037fc04f065fe03f037fb03f0ad
:020000040000fa
:2011a000e9f804f0f7fa04f061fc00f007fe00f0f9ff00004368064a591eff39914205d8e1
:020000040000fa
:2011c000da0703d5026895469e4670477047c04600ff1f000a4b0b4a596810b5914203d1c4
:020000040000fa
:2011e000094a9968914201d0012010bd00225a609a601b6818009342f7d0fff7dbfff3e752
:020000040000fa
:2012000000000020a5a55a5a3c3cc3c3044b054a18605a60044a9a60044b054ada6070470b
:020000040000fa
:2012200000000020a5a55a5a3c3cc3c300ed00e00400fa0570470e2010b501f06cf910b5fd
:020000040000fa
:2012400009490a4a0a4806f0e5f80021094a0a4806f0fbf80423094a91690b439361084b0b
:020000040000fa
:20126000084a9360fff77cff98ad00001c0000000c000020101d0000280000200004004072
:020000040000fa
:201280000010000000ed00e0044b98689b6880b25b035b0f033398407047c04600400041d9
:020000040000fa
:2012a00010b500f0a7ff0020fff7b0ff10bdf0b50e4b85b01d880e4b1e880e4b1f68fff794
:020000040000fa
:2012c000e3ff0d4b0d4cc01817230d4a0390019320002b000b490297009606f0cff80a490d
:020000040000fa
:2012e0000a4806f0cbf805b0f0bdc046b8100000d41a0020d40f002000f0ffff759a0000a5
:020000040000fa
:20130000509a00005d9a00006d9a0000109b000010b5092804d83030c0b200f057ff10bd83
:020000040000fa
:201320005730f9e710b504000134631e1878002800d110bd00f04afff6e7f7b50025174b28
:020000040000fa
:20134000174a1b78ab4200d8f7bd0026ab009b580193019af300d3181a68002a02d101359a
:020000040000fa
:20136000edb2ece75f683800fff7dcff380006f074f8431cff182d231c1a002c08d1380058
:020000040000fa
:20138000fff7d0ff01360a2000f020fff6b2e0e7202000f01bff013cefe7c0465c000020ca
:020000040000fa
:2013a0003000002070b5040000f048ff002802d02000fff7b7ff00222e4b2f4d1a7000f026
:020000040000fa
:2013c00019ff00f026ff0400152837d016d80a283ad00d2838d0082812d02a002d3213780b
:020000040000fa
:2013e0007d2becd8591c1170244ad45400f026ff0028e4d0200000f0e9fee0e77f28ecd1e2
:020000040000fa
:201400002b002d331b78002bd9d000f017ff002802d01b48fff786ff2a002d321378013bac
:020000040000fa
:201420001370cce700f00aff002802d01448fff779ff2a002d321378013b13702b002d335b
:020000040000fa
:201440001b78002beed1bae700f0f8fe002802d00a2000f0bbfe29000a202d310b78074a36
:020000040000fa
:201460002e35d054981c087000210133dbb22970d15470bd5d00002030000020900200206d
:020000040000fa
:20148000d4a000000a4b10b518001c000a2209492e302d340a7024780278944204d9541c9a
:020000040000fa
:2014a00004700548825c0a702f33187810bdc046300000205f0000209002002010b500f018
:020000040000fa
:2014c000a8fe03003038c0b2092806d91a00613ad2b2052a02d8573bd8b210bd1a00413ab9
:020000040000fa
:2014e000d2b2052a01d8373bf6e70122014b00201a70f2e76000002010b504000009fff7d7
:020000040000fa
:2015000007ff0f202040fff703ff10bd10b50400000afff7f1ffe0b2fff7eeff10bd054b26
:020000040000fa
:2015200001201b78202b02d0093b58425841c0b27047c0465f00002010b5fff7f0ff0028e3
:020000040000fa
:2015400000d110bdfff79efff7e7f8b51e48fff729fffff797fffff7efff1c4b1c4c1d7877
:020000040000fa
:20156000fff790ff0d2df1d00a2defd023002c331f78200000239f4204d123000222303339
:020000040000fa
:201580001a7019e0026894460022d10061440e68002e03d10133dbb20430ece7496809787a
:020000040000fa
:2015a000a94202d00132d2b2efe7b047230030331b78013b012bc9d80648fff7b3fe0023b0
:020000040000fa
:2015c00030342370c2e7c046b59e00005f00002030000020279b00000300303bdbb2092b52
:020000040000fa
:2015e00001d858b270470300613b052b02d8573840b2f7e70300413b052b01d83738f7e774
:020000040000fa
:2016000001204042eee7f8b5002406002500fff793ff0c4b0c4f1878fff7deff002809daae
:020000040000fa
:20162000e4b2002c01d0ff2e02d0012330373b702800f8bd2d0101340543fff723ffb4424c
:020000040000fa
:20164000e7d1f5e75f0000203000002010b50220fff7d9ffc0b210bd10b5ff20fff7d3ff87
:020000040000fa
:2016600010bd10b5fff7f8ff064b1b78002b07d1054a064b127812019b18421e9041187358
:020000040000fa
:2016800010bdc04660000020b5040020a4040020f8b5fff751ff114b00261b78104d2d2b99
:020000040000fa
:2016a00002d1fff7effe0136012200240a272b002f331b78303bd9b2092905d87c431c19ac
:020000040000fa
:2016c000fff7e0fe0022f2e7002a02d0012330352b70002e00d064422000f8bd5f00002023
:020000040000fa
:2016e0003000002010b504002278002a01d1012008e00749074b0978914204d00222002024
:020000040000fa
:2017000030331a7010bd0134fff7bcfeece7c0465f0000203000002010b5fff70dff08486b
:020000040000fa
:20172000fff7e0ff00280ad000f064fd642000f0d5fc044b044a0820da6000f0ecfe10bd96
:020000040000fa
:20174000359b000000ed00e00400fa0510b5064a064913780a2b02d9062000f0dcfe5c1c82
:020000040000fa
:201760009b001470585010bd5c0000203000002010b50448fff7eaff034a0449044800f043
:020000040000fa
:201780008dfb10bdd8a000003b9b00004b1500006800002010b502f068f8084b084c19687f
:020000040000fa
:2017a000206800f045fea8220649206800f0defd002004f083f902f057f810bdd00f002065
:020000040000fa
:2017c000d40f00201c03002070b500240c2632006243084bd558002d00d170bd280005f0ad
:020000040000fa
:2017e0003cfe01302a1829000348013405f046fee4b2ece768a100003f9b000010b5034bfb
:020000040000fa
:201800000348197805f03afe10bdc046bc030020499b000010b5034b0348198805f02efe09
:020000040000fa
:2018200010bdc046be0300205d9b0000044b10b599690448890a09b205f020fe10bdc04666
:020000040000fa
:201840001c0300206c9b000010b5034b0348597f05f014fe10bdc0461c030020839b0000d5
:020000040000fa
:2018600010b50b4c0b481223e25e0423e15e05f005fe23009e3300229b5e22009a349c3259
:020000040000fa
:201880000021525e0020215e034805f0f7fd10bd1c030020989b0000b39b0000f0b500254d
:020000040000fa
:2018a00080272b4b87b00100180005f0e7fd00f0a1fc00f0aefc274805f0f8fd00f09afcdc
:020000040000fa
:2018c000254805f0f3fd00f095fc244b02951b78019504930095ff003e00204800f060fbea
:020000040000fa
:2018e000049b03931f22039c1d4b60010593c018631c1a40194b37001b78013e0494039227
:020000040000fa
:20190000b6b2a342e8d001f0f1fa009b64011b180093059b019a1c19a38a1bb2d31a019335
:020000040000fa
:20192000638a029a1bb2d31a0293e38a1bb2ed18002ed7d1019a0b4b92121a80029aad1230
:020000040000fa
:2019400092125a809d80009b981200b207b0f0bdda9b0000ff9b0000029c00006815002047
:020000040000fa
:20196000400700201003002070b5fff7e5fd0d4b0c251c78fff786fd00230b4a28005843ff
:020000040000fa
:201980008158002903d10222084b1a7005e00978a14203d112185368984770bd0133dbb2a1
:020000040000fa
:2019a000ece7c0465f00002068a100006000002070b50b4c0b4800f0dbfee579002d04d04f
:020000040000fa
:2019c000fff7e8fe00230125e371a01d00f0eefe0548002d00d1054805f068fd70bdc046d0
:020000040000fa
:2019e0001003002016030020119c0000179c000010b5054c200000f0bbfefff7cbfe20005d
:020000040000fa
:201a000000f0d4fe10bdc0461603002070b5424e424800f0adfe357a002d7cd101f025ffe0
:020000040000fa
:201a20003f4c404ba8221868210000f02ffc2378012b0cd03c4b032229003c48236005f096
:020000040000fa
:201a400004fd06223a483b4905f0e4fca57165781a2d5ed003f020fe002d13d1257400233c
:020000040000fa
:201a6000a3806382c0239b02a36100232377002363770122631dda77102200212e4805f06e
:020000040000fa
:201a8000e4fc0be0012dead0032debd9042decd0052decd0072decd9082dedd0092d26d8a5
:020000040000fa
:201aa0006423a2795343254a9b18a3630023a38758220021224805f0c8fc230000229833ab
:020000040000fa
:201ac0001a80220000239a32138022009c321360a380638223005e22a0331a702300052213
:020000040000fa
:201ae000a2331a8023000022a4331a700de00a2ddcd00b2ddcd00c2ddfd00e2de1d90f2d04
:020000040000fa
:201b0000e8d0112dead9192decd91a236370193bf3710123337270bd1003002016030020d7
:020000040000fa
:201b20001c030020d40f00200100fa002903002023030020279c00004103002076a1060092
:020000040000fa
:201b40005c030020012310b50248c371063000f02dfe10bd1003002010b5fff799fd064bac
:020000040000fa
:201b600004001b78002b05d1fff750ff034b1c70fff7e8ff10bdc04660000020bc0300209f
:020000040000fa
:201b800010b5fff785fd064b04001b78002b05d1fff73cff034b1c80fff7d4ff10bdc04668
:020000040000fa
:201ba00060000020be03002010b5fff771fd124b1b78002b0bd1840204f042f9002807d0f0
:020000040000fa
:201bc0000e4b9b69a34202d00d4805f06ffc10bd0c4b1968a14204d2890a0b4805f04efcb9
:020000040000fa
:201be000f5e7fff713ff094b044a1b685b421c409461fff7a7ffeae7600000201c030020c2
:020000040000fa
:201c00002e9c0000d40f00205d9c0000d00f002010b5fff73dfd0c4b04001b78002b11d10f
:020000040000fa
:201c200001331c40fff7f2fe084b5a7fa24206d004215a5e598a5242494299805a825c77a1
:020000040000fa
:201c4000fff780ff10bdc046600000201c030020f0b587b0fff71cfd3d4c2378002b2bd147
:020000040000fa
:201c600005b2fff715fd002d28d12378002b25d038482570fff712fe374c05000022a35efe
:020000040000fa
:201c8000364800930222a35e012602930422a35e0493fff703fe07000022a35e01930222bb
:020000040000fa
:201ca000a35e03930422a35e0593bd4210db3a0029002b4805f0e2fb07b0f0bd002607b2f9
:020000040000fa
:201cc0002670059604960396029601960096ece7fff79cfe234ca5806782002e1fd0019b42
:020000040000fa
:201ce000009a9c466244d30f9b1822005b109a321380039b029a9c466244d30f9b182200c8
:020000040000fa
:201d00005b109c321380059b049a9c466244d30f9b185b109e342380fff714ffcce7fff70a
:020000040000fa
:201d2000b7fc0b4d2b78002bf6d123009a331880fff7aefc2b78002beed123009c331880c4
:020000040000fa
:201d4000fff7a6fc2b78002be6d19e342080e3e760000020739c000010030020769c000056
:020000040000fa
:201d60007b9c00001c03002010b5fff74ffe024800f01cfd10bdc0461603002070b5fff78b
:020000040000fa
:201d8000f3ff0b4b0b485a78197805f077fb00240c252a006243084bd158002900d170bd17
:020000040000fa
:201da0009b189b68002b00d098470134e4b2f0e71c0300209d9c000068a1000010b5024861
:020000040000fa
:201dc000fff7c4fc10bdc046e0a100004368026853601a6040600060704770b505000400d2
:020000040000fa
:201de00014352800fff7f2ff034b5a6863615d60a261156070bdc046c40300201c3010b557
:020000040000fa
:201e0000fff7e4ff054a0021100093680830834201d01c3b5968116110bdc046c40300205c
:020000040000fa
:201e2000f7b5eff31087019072b60f4eb46825681c3c1c3d3200230008321c33934203d087
:020000040000fa
:201e40006368019ad31a02d587f31088f7bd002320006360fff7d2ff2000fff7beffeb699e
:020000040000fa
:201e60002c001c3b1d00e5e7c4030020094b1a000832da609a6000225b601a611b60064b0f
:020000040000fa
:201e80001032013ad2b25b601b600833002af8d17047c046c403002024040020f7b5234dd5
:020000040000fa
:201ea00004002e7d01200192102e3ad100f033fb04cf127a824230d00133dbb29e42f7d1cc
:020000040000fa
:201ec000019b0026236189239b0020722660e150203b3100e018202205f0b7fa80239b0082
:020000040000fa
:201ee000e650043be6502300eff31086fd33ff33e360e93bff3ba361636108332362e361cd
:020000040000fa
:201f000072b62000fff769ff2b7d9a00aa18013394612b7586f31088f7bd0130c0b20028be
:020000040000fa
:201f2000ced02f0000231837c8e7c046c40300201a4ca36d002b0fd0ffb5eff3008001b47b
:020000040000fa
:201f4000eff3108001b46a46a36dda6028339a4202d20c2000f0dffa72b6a06d002804d02f
:020000040000fa
:201f60000368002b01d1fff738ff2368a3420ad123005c331b78002b02d062b672b6f4e724
:020000040000fa
:201f800030bf62b6fae7143ba365db689d4601bc80f3108801bc80f30088ffbdc4030020b9
:020000040000fa
:201fa000f8b5040072b6104fa406bd6d240f2e00143628603000fff709ff0c4be4001b1945
:020000040000fa
:201fc0005a685e606b61aa61eff31083166083f31088fff7adff0020bb6d1a68824202d0af
:020000040000fa
:201fe000186058600130f8bdc403002024040020f8b5124b05001b7d002b11d0eff3108671
:020000040000fa
:2020000083060f4a1b0fdb009f1872b6985804681438143c030014339f4202d186f31088f3
:020000040000fa
:20202000f8bd0368ab4203d100230360fff7d5fe63692000143b1c00ece7c046c403002059
:020000040000fa
:2020400024040020f7b50c1e01902dd0eff3108572b600f0a1fa1f4f631c1818ba6d00283e
:020000040000fa
:2020600000d101301c4ebb68b4461a4950601c3b1e001c36664505d110001c30cb68664641
:020000040000fa
:20208000c86008e05e68361a360420d410001b6a1c301e6870601362d66118608b681c3b47
:020000040000fa
:2020a0005b683b6185f310880198fff779ff0500002c0ad0eff3108472b6064b986d002388
:020000040000fa
:2020c0004360fff79bfe84f310882800febddb691c3bcde7c4030020cc030020010010b5f1
:020000040000fa
:2020e000002800d101310248fff7acff10bdc04621040020f8b572b6174e00253300327d71
:020000040000fa
:20210000b76d18336c1caa421ed138001430fff75dfe38001c30fff759fe337d0022013b41
:020000040000fa
:20212000dbb23375ab4202d35b1bdbb29a003000e1b218308900ad004118401905f073f9b7
:020000040000fa
:202140000023b365fff7f4fe0433191f0968b942dbd0e5b2d6e7c046c403002073b500f07d
:020000040000fa
:202160001bfa002405000c4b1a7da24200d873bda2009b189e697368317a3268002b09d0c7
:020000040000fa
:202180005b1b1bb2366905480096013405f076f9e4b2e8e7024bf5e7c4030020b49c00001c
:020000040000fa
:2021a0000f2700000022084b10b59a65eff3088383f309880223eff31482134383f3148837
:020000040000fa
:2021c000bff36f8ffff7b4fec403002070b50400054d0a2802d10d206b68984720006b686e
:020000040000fa
:2021e0009847002070bdc046a404002010b5fff7edff10bd034b10b59b68002b00d0984781
:020000040000fa
:2022000010bdc046a404002010b5fff7f3ff002010bd10b572b6064c23689847431c04d1ac
:020000040000fa
:2022200020001030fff7bcfef5e762b6c0b210bda404002010b5fff7ecff10bd014b187b41
:020000040000fa
:202240007047c046a4040020034b9a6001221860596000201a737047a404002010b501f07b
:020000040000fa
:2022600004fb064b0648196805f008f9054b0648196805f003f901f005fb10bdcc0f002080
:020000040000fa
:20228000d29c0000d00f0020e59c0000f8b505000f00140001f0e9fa114b1b68ab4201d802
:020000040000fa
:2022a0000020f8bd62199342fad3002c01d10120f7e70c4b1b885a1e2a409b1a1e1c9bb217
:020000040000fa
:2022c000a34200d9261cb6b232003900280001f091fa0028e4d0a41bbf19a4b2ad19e4e72d
:020000040000fa
:2022e000cc0f0020d80f0020f0b585b0fff7b4f91b4b04001d78002d2ed10227194b18008f
:020000040000fa
:20230000019300f035fa23020393174b80220293039b0299e818fff7b9ff002816d000249d
:020000040000fa
:20232000281980b2fff7f2f800262020fff74eff029b1b19985d0136fff7def8082ef4d1dd
:020000040000fa
:202340000a200834fff742ff802ce9d18025012f04d1019800f02afa05b0f0bd0127d4e7de
:020000040000fa
:2023600060000020b6040020b7040020f8b505000f00140001f079fa114b1b68ab4201d84a
:020000040000fa
:202380000020f8bd62199342fad3002c01d10120f7e70c4b1b885a1e2a409b1a1e1c9bb236
:020000040000fa
:2023a000a34200d9261cb6b232003900280001f0e5f90028e4d0a41bbf19a4b2ad19e4e7f9
:020000040000fa
:2023c000cc0f0020d80f0020f7b5070001f04dfa144b1800009300f0cbf9134b1d68002d42
:020000040000fa
:2023e00005d10124009800f0e1f92000febd2e00802d00d980260d4b38001900b2b20193aa
:020000040000fa
:20240000fff744ff041eedd00023019ad25cff2a05d101339e42f8d1bf19ad1bdfe7002452
:020000040000fa
:20242000e0e7c046b6040020d00f0020b7040020f8b5124f04003e68701e4018310003f059
:020000040000fa
:202440000ffe70430500a41b2418002d01d101200ee004262000fff7b7ff002809d1200096
:020000040000fa
:2024600001f054f9002803d0013e002ef2d13000f8bd3b68e41aed1ae7e7c046d00f002093
:020000040000fa
:2024800010b5fff759f80548fff72cf9002804d0034b00201968fff7cbff10bdfe9c0000b6
:020000040000fa
:2024a000d40f002010b5fff7d7f8054b1b78002b04d1044b00021968fff7baff10bdc04658
:020000040000fa
:2024c00060000020d00f002010b501f0f1f90248fff73cf910bdc04620a3000030b50425c4
:020000040000fa
:2024e000ff240138c0b22b000ee0c0460139c9b20029fad1013ad2b2002a01d02100f4e790
:020000040000fa
:20250000013bdbb2002b01d02200f7e70138c0b2ff28e8d130bdf8b5050072b640263f23dc
:020000040000fa
:2025200006401d401420fff7d9ff052401274b2001f0fefa3800fff7d1ff013c962001f06f
:020000040000fa
:20254000f7fae4b23800fff7c9ff002cefd1200001f0eefa0220fff7c1ff002e0bd04b20cd
:020000040000fa
:2025600001f0e6fa2820fff7b9ff200001f0e0fa0a20fff7b3ffac42d4d25e2001f0d8fa02
:020000040000fa
:202580000a20fff7abff002001f0d2fa01340a20fff7a4ffe4b2eee7014b18687047c046a8
:020000040000fa
:2025a0003805002070b50b4b0b4918688e681a689042fad10023094a002103f021ff14227a
:020000040000fa
:2025c0000d00040000233000002103f019ff0019694170bd3805002010e000e080969800a0
:020000040000fa
:2025e00010b562b6114b1b68db031dd5104c114a236812680133236023689b1a02d420683e
:020000040000fa
:20260000fff70efc23790c4a0133dbb2237111788b4209d11378002b06d00023237101f00f
:020000040000fa
:20262000ebf9201dfff7e4fc10bdc04610e000e038050020d40300201c000020eff31083fb
:020000040000fa
:2026400072b60021034a1070034a117183f310887047c0461c000020380500200022074bbd
:020000040000fa
:2026600007491a6059609a6007321a60c023054a1b06116a0b4313627047c04610e000e00c
:020000040000fa
:20268000ff52070000ed00e00223284830b542680124134343600c2325498a691343254a7e
:020000040000fa
:2026a0008b6114701378234203d053785bb2002bf8db214b214c1c6102241d692c431c6123
:020000040000fa
:2026c0000124dd682542fcd01d4cdc641d4c9c6400245c645d6c02342c435c6404241d6d87
:020000040000fa
:2026e0002542fcd002241d6d2542fcd0547864b2002cfbdb00249460547864b2002cfbdbe4
:020000040000fa
:20270000842464025460547864b2002cfbdb00220a724a728a72ca7202211a6a8a431a6291
:020000040000fa
:20272000802342681343436030bdc0460040004100040040000c00400008004044d30000f0
:020000040000fa
:2027400014007f00ff02000010b5027803008a4202d10320fff7dffeeff3108272b60478f6
:020000040000fa
:202760000020844201d11970013082f3108810bd70b50d4d02782b6804001b7a9a4202d139
:020000040000fa
:202780000320fff7c8feeff3108672b62378002b05d12b681b7a237086f3108870bd200005
:020000040000fa
:2027a000fff7fefbf2e7c0461c04002010b5094b02781b681b7a9a4202d00320fff7abfef0
:020000040000fa
:2027c000eff3108472b600230370fff711fc84f3108810bd1c040020e02110b5094bc900c3
:020000040000fa
:2027e0001a8c90b20a420cd01884830509d50f231840054bc100ca58002a02d05b185968da
:020000040000fa
:20280000904710bd004800414005002073b51e4c01002288238c656a92b200959bb21b48e2
:020000040000fa
:2028200004f02cfe1a4b1d68280004f01dfe20004030a16ae26a236b06781648009604f07e
:020000040000fa
:202840001dfe280004f010fe2300616c4e334f341a782378d2b2dbb20f4804f00ffe280081
:020000040000fa
:2028600004f002fe0d480188428843688468c66889b292b201960094094804f0fffd2800e4
:020000040000fa
:2028800004f0f2fd73bdc04600480041039d00001ca30000329d0000689d000060060020dd
:020000040000fa
:2028a000959d0000f7b508ac20cc009226880e4c0b9ac7000193e3195a600a9b3b510b4cc2
:020000040000fa
:2028c000019b07013e53e4196380009b6160a3600023e360064b1a003f32107002225d64dd
:020000040000fa
:2028e00040331a70f7bdc046400500206006002000480041034b1a003f32107000224033bf
:020000040000fa
:202900001a707047004800412022234b70b559690a435a611022d9690a43da610722596967
:020000040000fa
:202920000a4301215a619a690a439a61da690a43da611a6a0a431a620023184a1380118061
:020000040000fa
:20294000108803000b400842fad11549022451631449154d91633f211361917313491180cc
:020000040000fa
:202960000121134a0e1c2b70167010780842fcd110480133dbb204700c2bf4d14022c12022
:020000040000fa
:202980000d4b80001a6019580c4a1140c02292020a431a5070bdc0460004004000480041a0
:020000040000fa
:2029a00060060020a00500203f480041020f0000404800414d48004100e100e0ffff00ff96
:020000040000fa
:2029c000042370b50f268d001d40ae40aa404c080419303423784018b3431343dbb2237080
:020000040000fa
:2029e0000123403002789a431343037070bd012310b50348c9b243544018fff7f9fa10bda2
:020000040000fa
:202a000020070020f0b5072489b015000eaa12781c402c4b07000692a0000faa1278c058a2
:020000040000fa
:202a200072b60026284b1e55069bb34200d07f19002a00d049196600038df3b20793234b65
:020000040000fa
:202a4000d2020293092313439bb20193721c204b12022830134304900a00009301002b0092
:020000040000fa
:202a6000f0b20394fff71eff8022f3b201330593b31c1b0212041a43069b0092591e8b4122
:020000040000fa
:202a800080219b0249015b1800210391029101310b43019339002b00049a0598fff702ff49
:020000040000fa
:202aa0000948035d002b08d00598fff723ff0798fff720ff62b609b0f0bd0019fff770fa02
:020000040000fa
:202ac000eee7c046b0a3000020070020ef29000060008000204b8200d15802008023143288
:020000040000fa
:202ae000db0113431d4af0b5538053785bb2002bfbdb0124060025000936b540184a184ba3
:020000040000fa
:202b00001560b2109200d2181823c025f6001e40e733b340ad0057599f430423b340260002
:020000040000fa
:202b20003b435351831c9e4033000e4a156a2b4313620c600b682342fcd1cb692342f9d195
:020000040000fa
:202b4000094b01220b6080239b024b60074b40005242c252f0bdc046b0a30000000c00401c
:020000040000fa
:202b600000e100e0000400400c002000260700200823084a10b5d4692343d36101238b40cf
:020000040000fa
:202b80004622836183604018403003789343037010bdc046000400401300002213b5044c16
:020000040000fa
:202ba0000192013200920a002100fff72bff13bd320700201fb504000f2013000022684461
:020000040000fa
:202bc0000470044c019200920a002100fff71aff1fbdc046320700201300ff2213b5040097
:020000040000fa
:202be00005488274fe3a01920022123000920a002100fff707ff13bd2007002013b50124a6
:020000040000fa
:202c000001940094fff7fefe13bdf0b50726372585b0064001908748874c80190391fff7ca
:020000040000fa
:202c2000a7fd019bb2001d40844b0634d758730002931b5b9d4200d190e0052b38d011d84e
:020000040000fa
:202c4000002b1cd0032b28d07d4e052d00d1cee07c4c38d8002d5ad0032d00d1a4e00d20da
:020000040000fa
:202c6000fff759fc102befd1012377490a781a430a7076490a781a430a70754a09e00123ed
:020000040000fa
:202c800074490a781a430a7073490a781a430a70724a11780b431370d6e7012370490a78d7
:020000040000fa
:202ca0001a430a706f490a781a430a706e4af0e701236e490a781a430a706d490a781a43d4
:020000040000fa
:202cc0000a706c4ae5e7102dc9d104212000fff74fff05212000fff74bff0823f2695c49e7
:020000040000fa
:202ce0001343f361402363600a7807339a43453b13430b70032204212000fff761fe032236
:020000040000fa
:202d000005212000fff75cfe0322062120e008212000fff72dff09212000fff729ff0821d5
:020000040000fa
:202d2000f36947200b43f361802302264b4adb006360137883433343137020003200fff79e
:020000040000fa
:202d40003ffe320009212000fff73afe32000a212000fff735fe484b029a9d5280216b4676
:020000040000fa
:202d60008020019a8905d2050a4001999b8949054005bb8101403b680a4340490b40c021f6
:020000040000fa
:202d80001a43019b89021b020b40c0211a43019b89039b020b401343022213433b60fb692a
:020000040000fa
:202da0001342fcd105b0f0bd16212000fff7e0fe17212000fff7dcfe0823f26947211343f8
:020000040000fa
:202dc000f36180230226284a5b036360137820008b433343137031393200fff7f1fd32001d
:020000040000fa
:202de00017212000fff7ecfd2a001421b0e7244c16212000fff7bcfe17212000fff7b8fe2b
:020000040000fa
:202e00000822f3691b491343f361472362600a7820009a43453b13430b7003221621fff7d0
:020000040000fa
:202e2000cffd032217212000fff7cafd032211008ee7c0463307002020070020b0a30000e7
:020000040000fa
:202e4000000400400044004144440041454400414644004148440041494400414a440041e1
:020000040000fa
:202e6000564400415744004154440041d6440041d7440041c344004126070020ffffcccfdd
:020000040000fa
:202e800080440041072302211840074b8200d35810b51a688a431a60da690a42fcd1034b51
:020000040000fa
:202ea0001818fff783fc10bdb0a300003307002010b50020fff70efe0320fff70bfe0520c5
:020000040000fa
:202ec000fff708fe10bdc04610b5064b202219781f2301391940044b4901c91804f09afa63
:020000040000fa
:202ee00010bdc0463c07002040070020044b808a5b7f00b2002b01d0404200b27047c04663
:020000040000fa
:202f00001c0300207fb50c4c0a26a55f0422a35e0021625e0220215e02950626a55f5242ae
:020000040000fa
:202f20006d4201950825645f494264420094034804f0a4fa7fbdc046400b0020d99d000097
:020000040000fa
:202f400037b580256b46064ced0018715971054a6561022101a8fff71ffea56137bdc046a9
:020000040000fa
:202f6000004400410505000037b580256b46064c2d0118715971054a6561022101a8fff7d6
:020000040000fa
:202f80000bfea56137bdc0460044004105050000f7b56b460600d81d8023802715005b4245
:020000040000fa
:202fa0003343084c084e3f0103700091220077610121fff7f1fd290022000098fff70cfeca
:020000040000fa
:202fc000b761f7bd0505000000440041f7b56b4680270400d81d92230a4d0b4eff002a000b
:020000040000fa
:202fe000037001217761fff7d7fd6b462a00981d0121fff7f1fd2a0006212000fff7ecfdb4
:020000040000fa
:20300000b761f7bd050500000044004170b5802686b0ef216548fff7f8fdb6217e20fff741
:020000040000fa
:203020008fff634db6211420fff79efff6000320fff754f800206e61fff750f85b48ae617a
:020000040000fa
:20304000fff720ff5948ef21fff7dffd6b46981c802301210370554a03ac6e61fff79cfd8f
:020000040000fa
:2030600002212000514afff7b7fdae6163781e2b00d091e0012221000020fff789ff2378d7
:020000040000fa
:203080000f2b00d088e004217d20fff759ff0020fff724f803214120fff752ffac21402083
:020000040000fa
:2030a000fff74eff0020fff719f80d216d20fff747ff01ad0520fff711f82800fff786ff3a
:020000040000fa
:2030c00009216d20fff73cff0520fff707f82000fff77cff00216d20fff732ff0022ab5e5d
:020000040000fa
:2030e0000021625e9b1a334a934255dd02216b5e0220215e5b1a93424edd0422ab5e042160
:020000040000fa
:20310000625e9b1a2c4a934246dd01213c20fff72bff02266b46dd1c012229003c20fff7be
:020000040000fa
:2031200037ff2b783342f5d004221d001540134232d1a9214020fff703ff03214120fff7ef
:020000040000fa
:20314000fffe29000f20fff70fff06211020fff70bff1648fff796fe0425ef211348fff74d
:020000040000fa
:2031600054fd2000fff732ff1221062269440220fff70eff0d48fff785fe72b60c22210045
:020000040000fa
:203180000e4804f047f90e4a0e4813782b431370fef706ff62b6e0e704230b4a11780b434f
:020000040000fa
:2031a0001370074a11780b431370d2e7050500000044004154050000a9020000400b00202a
:020000040000fa
:2031c0003d0700203c05002082180020802270b50023082146200b24d2000133dbb2202bea
:020000040000fa
:2031e0001fd180220023082146200c2412010133dbb2202b24d18026194df6006e61fff780
:020000040000fa
:20320000cbf90400fff7c8f9001b0128fad9ae61144a15491548fef741fe1548fef796fada
:020000040000fa
:2032200070bd0a2bd9d1134deb690b43eb610c4b114d9a619a602b7883432b702300cce7b0
:020000040000fa
:203240000b2bd4d10b4deb690b43eb61044b0b4d9a619a602b7883432b702300c7e7c046d6
:020000040000fa
:2032600000440041fa9d00000d300000500b0020c8a30000000400404a4400414b4400412c
:020000040000fa
:2032800010b5064904228b5e00200a5e5b420220095e034804f0f2f810bdc046780d0020bc
:020000040000fa
:2032a000019e000010b50b210348fff7aefc8022024b52005a6110bdc3080000004400417a
:020000040000fa
:2032c000802210b5034b520003489a61fff7dafd10bdc04600440041c308000007b56b4644
:020000040000fa
:2032e00018715971fff7deff0221034a01a8fff753fcfff7e5ff07bdc3080000802370b519
:020000040000fa
:203300000400124d124eab71fff7ccff310030000722104bfff772fcfff7d2ff2b7aea79f5
:020000040000fa
:203320001b020d4913435bba5b182380ab7a6a7a1b0213435bba5b1863802b7bea7a1b028b
:020000040000fa
:2033400013435bba5b18a38070bdc046780d00207e0d0020c30800000080ffff37b50400b0
:020000040000fa
:2033600001210920fff7baff88256b461d71fff799ff01a902220800094bfff73ffcfff788
:020000040000fa
:203380009fff6b465a790123100018401a4202d1fef7a4fee9e72000fff7b0ff37bdc0462a
:020000040000fa
:2033a000c30800000023f7b5544c80210a206373fff794ff0120fef791feaf236a461370ff
:020000040000fa
:2033c000fff770ff4e4b022269466846fff716fcfff776ff6b465b784a4e303b012b07d968
:020000040000fa
:2033e0000823494a11780b43137032781343337027000a20fef772fe08210920fff76effa7
:020000040000fa
:203400000e370a20fef76afe3800fff7a7ff0a20fef764fe10210920fff760ff0a20fef7bd
:020000040000fa
:203420005dfe200025001430fff798ff0e23e25e1421635e1a35d218d30f9b185b10638395
:020000040000fa
:203440000223fa5e1621635e0a20d218d30f9b185b106b800423fa5e1821635e0121d21873
:020000040000fa
:20346000d30f9b185b10ab80fff738ff0e210b20fff734ff802701233f026373637b002b86
:020000040000fa
:2034800002d06846fff73aff6b4600229b5e00216a5e9b1abb4200db1c4b1d4a934200dabe
:020000040000fa
:2034a000130069460b806b4602215b5e0220295e5b1abb4200db154b934200da144b69461f
:020000040000fa
:2034c0004b806b4604215b5e0420295e5b1abb4200db0e4b934200da0d4b6a46938072b64f
:020000040000fa
:2034e00006226946200003f095ff08233278094813433370fef754fd62b6bfe7780d002086
:020000040000fa
:20350000c30800003d07002082180020ff7f00000080ffff3c050020f8b5002308208024c9
:020000040000fa
:20352000214a64035373214a214ed1690143d16120494c6047243578a543453c2c433470c0
:020000040000fa
:20354000d4691d4e0443d461802424048c618c6046243578a5433570d56909262843d061f5
:020000040000fa
:203560008020164dc003486188602878a04328708020134d40000133dbb2202b08d1114a59
:020000040000fa
:2035800011491248fef78afc1148fef7dff8f8bd082bf0d1d7693b43d361886188602b78c8
:020000040000fa
:2035a000a3432b703300e6e7780d002000040040544400410044004157440041564400418c
:020000040000fa
:2035c00048440041149e0000a5330000980d0020f0a30000f8b5812636010400012130005b
:020000040000fa
:2035e000fff713fb0623084d084f320028007c6101212b70fff7d0fa3000bc61fff742fcbd
:020000040000fa
:203600006b6823436b60f8bdc00f002080440041f8b58027184cff00636805003b4223d006
:020000040000fa
:20362000812001210001fff7f0fa81220523134e012177612000120123700127fff7acfa36
:020000040000fa
:203640008122390020001201fff7c6fa23783b42f6d180238120db00b3610001fff712fc8e
:020000040000fa
:203660006368074a1340636080202b0c63702b0ae570c000a370f8bdc00f00208044004168
:020000040000fa
:20368000fffbffff70b51e4ca368002b20d18120012100018026fff7b8fa81229f23194d9f
:020000040000fa
:2036a000f600012120006e6112012370fff774fa8122042120001201fff78efa8120ae61d0
:020000040000fa
:2036c0000001fff7dffb2378ff2b02d10023a36070bda3781a00113a0e2af7d8103b1a0042
:020000040000fa
:2036e00001239340802252022261074aa3601b04e3609b18636180235b002383e8e7c046b4
:020000040000fa
:20370000c00f0020804400410000fffff8b5194c0500e2680020aa422bd92369eb189a42db
:020000040000fa
:2037200027d326001a363000fff722f8fff7aaff2800fff76dff0500fff74cff8120d823ce
:020000040000fa
:20374000012100012370fff760fa81220a4f0421120120007d61fff71ffa8120bd61000162
:020000040000fa
:20376000fff790fb636830002b436360fff71ef80120f8bdc00f002080440041f7b51a4db3
:020000040000fa
:203780001400ea68070001910020ba422bd9e3199a4228d31548fef7ebfffff773ff38005b
:020000040000fa
:2037a000fff736ff0600fff715ff81200223012100012b70fff729fa81220d4f04212800e5
:020000040000fa
:2037c00012017e61fff7e8f98122210012010198fff7e2f98120be610001fff753fb03488f
:020000040000fa
:2037e000fef7e4ff0120febdc00f0020da0f002080440041f7b5194d1400ea680700019107
:020000040000fa
:203800000020ba4229d9e3199a4226d31448fef7affffff737ff3800fff7fafe06008120c1
:020000040000fa
:203820000323012100012b70fff7eff981220d4f0421280012017e61fff7aef98122210027
:020000040000fa
:2038400012010198fff7c8f98120be610001fff719fb0348fef7aaff0120febdc00f002086
:020000040000fa
:20386000da0f002080440041704710b5044c2000fef77efffff706ff2000fef797ff10bd69
:020000040000fa
:20388000da0f002070b5074d074c2800fef770fffff7f8fe2800fef789ffa168034803f0ef
:020000040000fa
:2038a000edfd70bdda0f0020c00f00201c9e0000802230b50023082146200b24d2000133d1
:020000040000fa
:2038c000dbb2202b00d130bd0a2bf8d1064deb690b43eb61054b064d9a619a602b78834312
:020000040000fa
:2038e0002b702300ebe7c0460004004080440041ca440041024a537e5bb2002bfbdb7047b8
:020000040000fa
:2039000000400042054a064b12789a5c054b1343054a1361022313737047c046db0f00202a
:020000040000fa
:2039200018a400000018000f0040004210b58ab002ac2000fff7c8fa0622a35e0421625e8f
:020000040000fa
:203940000821615e03480091029903f097fd0ab010bdc046379e0000f7b51e4e1e4c3378f2
:020000040000fa
:2039600022781e495201488b5900521801331c49dbb288523370032b02d8fff7c3fff7bd46
:020000040000fa
:203980000122184b19780a431a7022781b78d2b200920d2b1bd1144b5701dd1928000622d5
:020000040000fa
:2039a00012490c30019303f035fd28000c221049123003f02ffd0f4b019a1b682000bb5004
:020000040000fa
:2039c0001f22009b013313402370fef711fb01237370d4e7db0f00203c070020004000423f
:020000040000fa
:2039e000440700203d07002040070020780d0020400b00203805002010b5054b5a78002a13
:020000040000fa
:203a000004d000225a701a70fff77cff10bdc046db0f0020384a394b70b5538053785bb238
:020000040000fa
:203a2000002bfbdb80230124354a364d116a5b020b4313622c70fff75dff2b782342fad15f
:020000040000fa
:203a40006b7e5bb2002bf6db2f4b0226186a596a196a5a6a5301ca0e1a43d2b22a85fff794
:020000040000fa
:203a600049ffe023db00ab80fff744ff1f23eb70fff740ff6e70fff73dff8023c521234ae4
:020000040000fa
:203a80001b04ec7589002e701360535820481b021b0a5350fdf75afe0f211e4a1e4813783f
:020000040000fa
:203aa0008b432343137046220378a343234303700378934333430370184803788b43234364
:020000040000fa
:203ac000037017480378a343234303700378934333430370134803788b43234312490370c8
:020000040000fa
:203ae0000b78a34323430b700b7893431e430f4b0e705c7070bdc046000c00401e40000041
:020000040000fa
:203b000000040040004000420060800000e100e01ca400003144004142440041b4440041c8
:020000040000fa
:203b2000c8440041b1440041c2440041db0f0020044b002804d00222800118641a60704714
:020000040000fa
:203b40001860fce70028004210b50c00fff7f0ff2000fef7c3fa0022014b1a6010bdc0465d
:020000040000fa
:203b6000002800421b4a1c4b10b5538053785bb2002bfbdb80231949db000a6a13430b6287
:020000040000fa
:203b80000123174a136010681842fcd1906804001c401842f7d1bc2040011064d463937742
:020000040000fa
:203ba0000822c8690f4c0243ca61802146200e4a4902516191600d4a1178814311700f213d
:020000040000fa
:203bc000207888430b3901432170117899430b43137010bd000c00401b400000000400407b
:020000040000fa
:203be00000280042384400410044004150440041044b1a78012a03d8511c19700133985447
:020000040000fa
:203c00007047c046e00f0020f0b5224bda78002a16d000200125844619795a799f79dc7982
:020000040000fa
:203c20001d4e91421cd12200e81bc0b202412a4209d16246002a03d09f71dc7159711971e3
:020000040000fa
:203c400001204042f0bd2a0082409443020008321201b21852680700ac460021d2b2e0e719
:020000040000fa
:203c60006046002802d09f71dc715a714d1c9c79edb21d71094ba0011b18585caa42e1d157
:020000040000fa
:203c800001230634a340c2220549dbb252008b54d8e7c046e00f0020541100205410002016
:020000040000fa
:203ca0000050004170b50d4b0d4d5b682a7a9b049b0c1c1c934200d9141c2900ee68a4b204
:020000040000fa
:203cc000121b2a7230002200103103f0a3fb4022044b3619ee605a7170bdc0465411002026
:020000040000fa
:203ce000e00f0020ff500041f8b5124ef3795bb2002b1edb104d20242b781f2b04d82a00e7
:020000040000fa
:203d000000211c003032117028006f6b1b1b2200390038302b7003f07dfb084a3f1953691c
:020000040000fa
:203d20006f631b0f1b071c4380235461b371783b3372f8bdff500041e00f00205411002059
:020000040000fa
:203d400010b501240548064a037812781341234200d110bdfef724f9f4e7c0463810002025
:020000040000fa
:203d600039100020012030b5194a1a4b117802001c008a40583425782a4322701a005a32cd
:020000040000fa
:203d80001478402c02d01a005b3210700800124a0a30000112185068a625000f0007044389
:020000040000fa
:203da000546001221400881d8440e0b20b4cff3560551500881c8540e8b2a825ff3560550f
:020000040000fa
:203dc0001800521a5930027000225a331a7030bd39100020e00f00205411002000500041b0
:020000040000fa
:203de00010b5094ce378002b0cd072b65b342378002b06d1fff7a4ff2378002b01d1fff7cc
:020000040000fa
:203e0000b1ff62b610bdc046e00f002070b5114c0500e378002b1bd072b6fff791ff23002f
:020000040000fa
:203e200000225b331a7023005a34593320781978094b421c8901d2b25b1822701d54402a42
:020000040000fa
:203e400001d1fff78fff62b60a2d01d1fff7c8ff70bdc046e00f0020d41000200120f0b522
:020000040000fa
:203e6000c54d85b0ab8b9bb202932b8c9ab20392029aaa8303427cd0c04ac149137a022628
:020000040000fa
:203e8000dbb21372bf4c0a78df0600d4bbe002430a70334205d0220004235c3211780b4378
:020000040000fa
:203ea000137023005c331a78019200221a700123019f019a1f401a4230d0260007335e36ee
:020000040000fa
:203ec0002372e660fff7eefe237a002b26d10022b2563378002a03dbf288002a00d00227ec
:020000040000fa
:203ee000220030321770621c626300221800227060321040134200d18ae0202800d165e1d7
:020000040000fa
:203f0000a14aa04b1278012a08d11a005e32d2881978914200d91a70fff7e6fe019b9b075a
:020000040000fa
:203f200011d5994e974c3378022b0cd1fff7bafe237a002b07d1012232702278002a00d075
:020000040000fa
:203f40002370fff7d1fe019b5b0712d58e4b8d4c1b78012b01d1fff7c7fe220067321378e0
:020000040000fa
:203f6000002b06d08021663423780b43ab7200231370039bdb0612d58822ff32ab5c0321ed
:020000040000fa
:203f8000dbb2ab541a000a400b4208d07d4b7f48d9790a43da710122da70fef729f8039b72
:020000040000fa
:203fa0009b0610d5a822ff32ab5cdbb21900ab54a53aff3a1140134205d0754803788b433b
:020000040000fa
:203fc0000370fef715f8029b1b071ad56d4b714a714918001160802138308905516010614f
:020000040000fa
:203fe00051611121654a5170ee315171ec399172190000223031da700a705a631a70da6083
:020000040000fa
:204000001a7205b0f0bd034200d142e732433fe71f221340012b00d1a5e0022b00d1c9e01b
:020000040000fa
:20402000002b00d06ce723005e335878092800d966e702f00bf8c40065ff65ff65ff65ff0e
:020000040000fa
:204040000a00140065ff34003700220023005e32528866331a7001236734237050e72300f5
:020000040000fa
:204060005e3359884d4a0e0af7b2c9b21378002b00d145e75078b8420fd1481ec0b20029a5
:020000040000fa
:204080000ad1022e00d1937821005e31c988994200d2cbb26263e0e70100d218e6e768342e
:020000040000fa
:2040a000207890e023005e335b883d4a002613702200384b6c321e625e621a63902240211e
:020000040000fa
:2040c000ff2752005e63a9540432af542a220221ff32a954334a191dca671900c0221800dd
:020000040000fa
:2040e00092050831ca67304990300160190094310a60c02153204900685404316f545f3fee
:020000040000fa
:20410000bc468a2103209c446746ff316854274902383960b027bc4619009c446746a431bf
:020000040000fa
:204120000a602349b43339601a60d0233522ff275b00a071ea540433ef54aa230322ff33f7
:020000040000fa
:20414000ea54230059331e7023005b331870200058300670fdf74cff114b0c48e6711e70b9
:020000040000fa
:20416000fdf746ffcce65e346378002b27d00a2b00d0c5e627e0c04600500041ff500041e7
:020000040000fa
:204180003c100020e00f002010100020b40400203810002054110020f00f0020be100000b2
:020000040000fa
:2041a000481000205410002094100020d4100020141100205e346378002b00d0a0e60020e8
:020000040000fa
:2041c000fff716fd0020fff713fd99e623005e335b78202b06d0212b00d091e6044b6363e1
:020000040000fa
:2041e00007233ae7024be3600723237288e6c0462000002010b572b6fff706fd431c02d05a
:020000040000fa
:2042000062b6c0b210bd0248fdf7cafef4e7c046b404002072b68022084bda67084b7f3a1e
:020000040000fa
:2042200019890a4302211a811a788a431a70054a1e31d3698b43d36162b6704704e100e078
:020000040000fa
:204240000050004100040040f8b508233e490f25ca693e481343cb61062302783c4caa43a3
:020000040000fa
:2042600013430370012322789a431a432270602204782c4022430270364802789a4313437f
:020000040000fa
:204280000370354a354b538053785bb2002bfbdb2023ca69324c13430122cb612378134376
:020000040000fa
:2042a000237023781342fcd10125a378190029402b42fad180222b4e5200300003f0c5f866
:020000040000fa
:2042c0002389294a1d4325816662106a516a8b03db0e1f2b00d11a3b106a516a4902c90e7e
:020000040000fa
:2042e0001f2900d10239166a576aba01520f072a00d1043a9b010b431203134323850f239e
:020000040000fa
:20430000e37072b60023238106332370043ba2781a42fcd18023c1208021144a8000136097
:020000040000fa
:20432000135889041b021b0a0b4313500823238362b60f4bc046013b002bfbd10122238947
:020000040000fa
:2043400093432381f8bdc046000400403c4400415844004159440041000c004006400000d6
:020000040000fa
:2043600000500041541100200060800000e100e050c3000010b5fff767ff0022034b044995
:020000040000fa
:204380001a700448044afdf75fff10bd101000200d3e0000093c0000e13d0000042370b5a0
:020000040000fa
:2043a0000f268d001d40ae40aa404c080419303423784018b3431343dbb22370012340303e
:020000040000fa
:2043c00002789a431343037070bd0b4b00b598420ed10800183807280ad801f02dfe04043f
:020000040000fa
:2043e0000904070907070c39c8b200bd1439fbe70f200840f9e7c0460044004110b51c2400
:020000040000fa
:20440000c30880002040153c8440054a9b009b189a69a2430324214081401143996110bdf3
:020000040000fa
:2044200000180040f8b500240127084d2e693b00a340334206d0064a2b61e300d358002bc1
:020000040000fa
:2044400000d098470134102cf1d1f8bd0018004054120020f7b51500019307000c00fff789
:020000040000fa
:20446000b4ff194bc200d358002b02d01020fef752f801230826a340144a3c19d169314336
:020000040000fa
:20448000d1617b6069060fd50223403422789a431343237072b60c4b0199c200d15029009e
:020000040000fa
:2044a000fff7acff62b6f7bd0222002d03d0012d08d1bb6106224721403423788b431a437e
:020000040000fa
:2044c0002270e7e77b61f5e7541200200004004010b51400fff779ff72b62100fff78effe7
:020000040000fa
:2044e00062b610bd10b51400fff76fff72b6024bc000c45062b610bd54120020f8b5050034
:020000040000fa
:204500000c00fff762ff72b6012686400f4ffb681e4212d10423a2001a406308eb1830332b
:020000040000fa
:2045200019780b4bc00018180f2393400b40134103712b1940331b78437100222100280023
:020000040000fa
:20454000fff72cfffe6062b6f8bdc046001800405412002070b504000d00fff736ff72b6a2
:020000040000fa
:204560000122110081400a4bc0009960094b1b185979114206d0290020001a79fff70effd7
:020000040000fa
:2045800062b670bd6419403423781a432270f7e700180040541200200e4a0f4b10b5538055
:020000040000fa
:2045a00053785bb2002bfbdb01220c4b1a705a7852b2002afbdb1021c124094aa4001160ca
:020000040000fa
:2045c0001059ef318843fc390143115102221a7010bdc046000c0040054000000018004042
:020000040000fa
:2045e00000e100e0044b10b55843044b0449c01801f0c0fd00b210bd5f100000f2d7000072
:020000040000fa
:20460000e5af0100c343f0b50400002587b0db171c4003ae20000a2101f092fe2f002000e0
:020000040000fa
:20462000f1550a2101f0a6fd01350400edb20028f0d1154bf6190093144b0193009b347877
:020000040000fa
:20464000013da0331878edb2002c0fd01427013ce4b2019b39001878013cfff775fae4b264
:020000040000fa
:204660003800fdf73bfdff2cf3d105e03221fff76bfa1420fdf732fd1e20fdf72ffd013e60
:020000040000fa
:20468000002ddbd107b0f0bd1c030020bc030020f8b500249626234f234d200000f096feac
:020000040000fa
:2046a000012836d13b00a03318780221fff74cfa1420fdf713fd002c29d001f0c8fb002894
:020000040000fa
:2046c00024d00a20fdf70afd02260a243d009623a03528785e21584301f04cfd2100c0b219
:020000040000fa
:2046e000fff732fa21002878fff72efa4b202b785e21584301f03efd2100c0b2fff724fabe
:020000040000fa
:2047000021002878fff720fa012e09d1f8bd0124c3e728785e21704301f02cfdc0b2c4e732
:020000040000fa
:204720000126d3e71c030020bc030020f0b589b0304c314e23783370002b20d16846fef7a4
:020000040000fa
:20474000c3fb6b460820185e002803d12b48fdf727fcf3e7fff746fffff754ff3378092b89
:020000040000fa
:2047600005d1274b1878002801d0fff74bff3378082b20d1fa204000fdf7b0fcd8e7214a35
:020000040000fa
:20478000d75c002fead007253d40013dedb2ff2d03d12420fdf7a2fce0e71b4b14211878af
:020000040000fa
:2047a00008231f4200d10621fff7cef90620fdf795fc7f08e9e7012b01d1fff769ff322701
:020000040000fa
:2047c0002378022b07d0327823789a42b0d12000fdf7e6fbf7e7fff75bff3d002378022b70
:020000040000fa
:2047e000eed1013d0a20edb2fdf778fc002df5d1e6e7c04680180020d81200206815002066
:020000040000fa
:204800008218002049a40000bc03002010b5034a03490448fdf742fb10bdc0465b9e00006b
:020000040000fa
:204820002d470000e0120020134b04215a5e196852181a600c215a5e996852189a601421d3
:020000040000fa
:204840005a5e196952181a611c215a5e996952189a6124215a5e196a52181a622c215a5e72
:020000040000fa
:20486000996a52189a6234215a5e196b52181a63da8e0132da86704708150020074b10b551
:020000040000fa
:2048800038229c5e00220648510001324452402afad100223a331a7010bdc04608150020dc
:020000040000fa
:2048a00078150020f7b5164ca06c676c011c02f00dfa391c0190381c02f008fa011c019864
:020000040000fa
:2048c00002f044fb266c071c311c301c02f0fef9011c381c02f03afbe56b061c291c281cdd
:020000040000fa
:2048e00002f0f4f9011c301c01f084fe04f0a6f8044902f0ebf902f0effc2087f7bdc0460a
:020000040000fa
:2049000008150020e12e654270b514000d0004f0f1f92860011c02f0d9f9011cfe20800557
:020000040000fa
:2049200002f014fb04f034f8206070bdf0b54b6885b001938b680f680293cb6805000c0045
:020000040000fa
:20494000381c391c039302f0c1f90199061c081c02f0bcf9011c301c01f04cfe0299061c84
:020000040000fa
:20496000081c02f0b3f9011c301c01f043fe0399061c081c02f0aaf9011c301c01f03afed1
:020000040000fa
:204980000021061c01f008fd00281dd0301c03f0ffff011cfe20800501f0ccff391c041c9b
:020000040000fa
:2049a00002f094f901992860201c02f08ff902996860201c02f08af90399a860201c02f0ba
:020000040000fa
:2049c00085f9e86005b0f0bd2b0007cc07c322681a60f7e76e4bf0b51c001e001d001968cf
:020000040000fa
:2049e0006c4a49121180002299684e344912218019695036491231809969523549122980d3
:020000040000fa
:204a0000196a89b05965996a1a609965196b9a601a619a611a629a621a63d965fff72eff57
:020000040000fa
:204a20000023f05e5c4b5d4f00229b5ec01a02f073fc061c0023e85e3b009e3300229b5eaa
:020000040000fa
:204a40003d00c01a02f068fc071c0023e05e2b009a3300229b5ec01a02f05efc002304a95c
:020000040000fa
:204a600007900800049305960697fff75fff6b7f002b00d188e04a4c079b0021181c029304
:020000040000fa
:204a800002f024f9069f051c391c201c02f01ef9011c281c02f05afa059e0090311c201c44
:020000040000fa
:204aa00002f014f9291c02f051fa00210190381c02f00cf900210390301c02f007f9061c64
:020000040000fa
:204ac000011c039802f042fa0099071c081c02f0fdf80199051c081c02f0f8f8011c281c07
:020000040000fa
:204ae00001f088fd391c051c381c02f0eff8011c281c01f07ffd03f04bff311c051c039889
:020000040000fa
:204b000001f078fd0299061c201c02f0dff8011c301c01f06ffdfe218905041c01f06afd82
:020000040000fa
:204b2000fc21890502f0d2f803f032ff061cfe20211c800502f00afafc21890502f0c6f897
:020000040000fa
:204b400003f026ff291c01f0f5fe051c011c009802f0bcf80e4c291c2064019802f0b6f83c
:020000040000fa
:204b6000291c6064381c02f0b1f8a06420003c300100e663fff7dafefff794fefff77efe9b
:020000040000fa
:204b80000023e38609b0f0bdfe24a40574e7c0460815002054150020b80300201c03002017
:020000040000fa
:204ba000000080bff0b5cf488fb0fdf721face48fdf7f6f9cd4ccb4b26001d78ca4b683616
:020000040000fa
:204bc0001b789d4205d1307843425841c0b20fb0f0bdc74b6d01ea58ed1828006266fef73d
:020000040000fa
:204be00085f9ab8aa0805b42a3816b8a5b42a382eb8aa3832b8b5b42a384ab8ba3856b8b01
:020000040000fa
:204c00005b42a3863378002b1ed08023e28e9b009a4208d2fff708fe1f21b24a13780133af
:020000040000fa
:204c20000b401370c6e7b34bb348598a9b88c91a230009b26a33198001f09cfae066fff740
:020000040000fa
:204c4000c9fe00233370e7e7ac4b1b78022b0cd88022e38e9200934200d339e1fff7e4fd20
:020000040000fa
:204c6000e38e9b0601d100f075f900f08df92c23e05ea36d4002c01a02f04efbec218905ed
:020000040000fa
:204c800002f024f89e4902f021f89e4902f01ef8061c3423e05ee36d4002c01a02f03cfbd9
:020000040000fa
:204ca000ec21890502f012f8954902f00ff8954902f00cf8051c2423e05e636d4002c01a20
:020000040000fa
:204cc00002f02afbec21890502f000f88c4901f0fdff8c4901f0faff09aa08a9fff714fe4b
:020000040000fa
:204ce000301c0baa0aa9fff70ffe0daa281c0ca9fff70afe099b0b9d181c291c049301f002
:020000040000fa
:204d0000e5ff089f0a9e0d9b311c0690381c019301f0dcff0c9b019907900698029301f025
:020000040000fa
:204d2000d5ff02990390079801f0d0ff011c039801f060fc391c0390281c01f0c7ff311cdd
:020000040000fa
:204d4000051c049801f0c2ff291c061c019801f0bdff311c071c029801f0b8ff011c381c14
:020000040000fa
:204d600002f0f4f8311c0490019801f0afff291c061c029801f0aaff011c301c01f03afc11
:020000040000fa
:204d800002990590069801f0a1ff0799051c019801f09cff011c281c02f0d8f8e36b0399c1
:020000040000fa
:204da0000193236c06900198029301f08fff0499071c029801f08aff011c381c02f0c6f898
:020000040000fa
:204dc000656c0599071c281c01f080ff011c381c02f0bcf8a66c0699071c301c01f076fff0
:020000040000fa
:204de000011c381c02f0b2f80399e063029801f06dff0499071c019801f068ff011c381cae
:020000040000fa
:204e000001f0f8fb0599071c301c01f05fff011c381c01f0effb0699071c281c01f056ffba
:020000040000fa
:204e2000011c381c02f092f803992064281c01f04dff0499071c301c01f048ff011c381c2f
:020000040000fa
:204e400002f084f80599071c019801f03fff011c381c01f0cffb0699071c029801f036ffad
:020000040000fa
:204e6000011c381c01f0c6fb03996064301c01f02dff0499061c281c01f028ff011c301cc2
:020000040000fa
:204e800001f0b8fb0599051c029801f01fff011c281c02f05bf80699051c019801f016ff01
:020000040000fa
:204ea000011c281c01f0a6fba06420003c300100fff73cfdfff7f6fc21003a310b78124aec
:020000040000fa
:204ec000248f580084523f22013313400b70a3e68022d200934202d20133e386c0e6fff7af
:020000040000fa
:204ee00079fdbde6681500203c07002008150020400700201c03002014d0390180180020e0
:020000040000fa
:204f00006fa18b3a0ad7a33b7815002010b5fcf72bff00230d4ce3862360a380a36023615c
:020000040000fa
:204f2000a361a381a382a3832362a3622363a384a385a3862387fff7a1fc054b1a78230034
:020000040000fa
:204f400060331a7001236834237010bd081500203c07002070b50b4eb268f368b469f56906
:020000040000fa
:204f600030687168801a994132697369121bab413060716032617361b060f160b261f3612c
:020000040000fa
:204f800070bdc046f8150020f0b54c4e87b0706a00234b4ac11701f033fa346a0322e517f4
:020000040000fa
:204fa0000023009001912000290001f029fa009a019b12184b41306871681f0712093a4334
:020000040000fa
:204fc0001b1112184b41200000920193290000233b4a01f015fa3269736980185941b36a12
:020000040000fa
:204fe000f46a0290039104930594364b04229a5e354b00215b5ed21a344b1b6853431c0064
:020000040000fa
:20500000dd17049a059ba41a9d412b04240c1c43e517610feb000b43e200009801998018b3
:020000040000fa
:20502000594102000b00009001913260736020000023274a3463290001f0e2f9029a039bc8
:020000040000fa
:2050400012184b412000029203933261736129000023204a01f0d4f9049b059cc0186141bb
:020000040000fa
:20506000019bb062f1621c04009b000c1b0c1c43039b74631a04029b1b0c134373620b0451
:020000040000fa
:205080001843b36b30629c4200ddb463b36c1800d917326c736c121a8b412000e117121855
:020000040000fa
:2050a0004b413f2000213264736412184b4111005b06ca091a43b26407b0f0bdf815002078
:020000040000fa
:2050c0008f0200001c0300200c150020741500207f0200007c0c000010b50c244443064b40
:020000040000fa
:2050e000e418200002f0b9f9044a21001218044802f0c4f910bdc0468ca40000af9e00000c
:020000040000fa
:20510000629e0000012270b5040002231440104201d00e4a936105001d40184203d080222a
:020000040000fa
:205120000b4b92009a610b4b1888fcf7d7ff002c02d00222054b5a61002d03d08022044baf
:020000040000fa
:2051400092005a610520fcf7c9ff70bd0044004180440041be030020f8b505000688002e1c
:020000040000fa
:2051600001d101204ee074423440802c00d173e014d8082c0ad8002c0ed0601e07280bd878
:020000040000fa
:2051800000f05aff39410a480a0a0a4c202c4dd0402c4fd0102c45d0a643e0e780231b01dc
:020000040000fa
:2051a0009c4200d178e015d880239b009c4265d08023db009c4200d169e080235b009c4258
:020000040000fa
:2051c000ead1fdf7e9f93e4b1b68c01a6b69984217dce1e78023db019c4262d080231b02a0
:020000040000fa
:2051e0009c4265d080235b019c42d5d1354b1a8822216b5e03e00223ea5e334b1b689a42be
:020000040000fa
:20520000cada0020f8bd0423ea5e2f4b1b689a42f7dcc1e70623ea5e2c4befe70823ea5e21
:020000040000fa
:205220002a4bf3e70a23ea5e294be7e70c23ea5e274bebe7274f0022bb5e01225100795ab5
:020000040000fa
:20524000081c09b2994200da181c013203b2402af4d10e216a5ed2e71e4f0022bb5e0122f4
:020000040000fa
:205260005100795a081c09b2994200da181c013203b2402af4d110216a5ec8e7fdf78cf90a
:020000040000fa
:205280000f4b1b68c01aab699842badb84e70f4b1b68002bb5dd7fe70c4b1b68002bb0dada
:020000040000fa
:2052a0007ae70d4b6a1cd27f1b789a42a9d973e7094baa1cd27f1b789a42a2d86ce7c04666
:020000040000fa
:2052c00088180020a0180020181600201c1600202c1600207815002080180020f0b585b0f5
:020000040000fa
:2052e000fcf742fd364b03931b78022b3cd9354c0a212000fcf7a6fe039b1b78072b56d89c
:020000040000fa
:2053000000231d00304e271d02930193e289a3891343029a13410122134237d13388002b1f
:020000040000fa
:2053200034d03b68002b14d13000fff715ff00282bd080223388920113421cd0f569eb439c
:020000040000fa
:20534000db171d40fdf728f92d18002d00d101353d603000fff700ff00282ad0fdf71cf983
:020000040000fa
:205360003b68c01a0ad510e00398fcf719feb9e701230293cae73b68002bead10123029ae9
:020000040000fa
:205380009340019a1a4393b201930125029b04372c36002becd0019b002b06d0a389019abe
:020000040000fa
:2053a00013431000a381fff7adfe002d9fd1fcf7a1fe01230299e2898b401343e381e4e719
:020000040000fa
:2053c00080180020481600205c03002030b5eff31085040089b072b66846fdf775fd85f3cb
:020000040000fa
:2053e0001088640023006b440421595e6b4608229a5e084b03209a420addd310994207db57
:020000040000fa
:205400000f23534301201b11994200dc0020c0b209b030bde903000070b50020fff7d6ff8c
:020000040000fa
:20542000084d094c800042590021200002f026f80120fff7cbff800042590121200002f026
:020000040000fa
:205440001df870bdbca50000679e0000f7b50221214802f013f80023204e002501932048bd
:020000040000fa
:20546000019902f00bf83388ab421dd11d4802f01df8019b2c36002b00d0f7bd0123ece7f7
:020000040000fa
:2054800033883b420ed02800fff726fea379ff2b1ed08022f318d201974210d31978124859
:020000040000fa
:2054a00001f0ecff0135edb20c236b430f4ce418a788002fe4d10a2001f0f0ffd9e78c227c
:020000040000fa
:2054c0009201174201d01968e9e70021595ee6e7074801f0d3ffe5e77f9e00005c0300209f
:020000040000fa
:2054e0008f9e00009a9e0000a59e00008ca40000ab9e0000f0b591b0fcf71ef8534b00936b
:020000040000fa
:205500001b783f2b1dd100240c2611e02000fff7e3fdab794e48ff2b00d14e4801f0aeff7a
:020000040000fa
:2055200033006343fb18986801f0c0ff0134e4b235006543484f7d19ab88002be6d111b024
:020000040000fa
:20554000f0bdfcf7a5f8454b0290197801930029f5d10300012804d91900414801f08effaf
:020000040000fa
:20556000ede705ac2c22200001f06ffffbf7e4ff009b1b780a2b56d00025eeb2fbf7cffff6
:020000040000fa
:2055800000280bd1009b1b780a2b07d004aa53550135fbf777ff032defd10326002504abec
:020000040000fa
:2055a0009d552d4b03930c276f43039bdf19be88002e07d12b4804a901f060ff0223019af4
:020000040000fa
:2055c0001370bce7380004a901f01aff002802d00135edb2e7e72388bf7933432380ff2fef
:020000040000fa
:2055e000c4d0fbf7a9ff009b01251b782d2b02d1fbf748ff023dfcf74bf8019b45431b7899
:020000040000fa
:20560000002b9cd18023db019e4203d3002dd5dbe555abe78c239b01e7191e4201d03d60fb
:020000040000fa
:20562000a4e73d80a2e7fcf7f1f92c22029b5a430d4bd218130023cc23c307cc07c307cc9a
:020000040000fa
:2056400007c306cc06c3fcf77dfa78e75f000020b39e0000ae9e00008ca400006000002050
:020000040000fa
:20566000b89e0000d29e00005c03002010b504000748210001f002ff012c03d90222054b3d
:020000040000fa
:205680001a7010bd0120a04080b2fff73bfdf8e7e99e000060000020f0b5374b91b05b7831
:020000040000fa
:2056a000182b5ed810223548354901f0b3fe02230293013b009305ac04ab2a220021981d97
:020000040000fa
:2056c00001f0c3fe009b2f4a5b019918d35a80272380002301932c4b2c489c460391ff0168
:020000040000fa
:2056e0008379ff2b23d0002582886646a9008e5b96423ad16144cd78039e89787118082df7
:020000040000fa
:205700000cd0202d2fd00025495fba4209d300290ddbe1540be001230293cde70978ba42a1
:020000040000fa
:20572000f7d28c25ad01e3182a4223d01960019b0c3001330193112bd2d12c21009b2200e5
:020000040000fa
:205740005943134bc9180b0061ca61c323ca23c323ca23c303ca03c300230093029b012b5c
:020000040000fa
:20576000d9d111b0f0bd0968cfe701350e2dbcd10021d4e71980dae71c030020b4030020a0
:020000040000fa
:205780009a0300205a03002054a400008ca400005c0300200821022010b546240e4ad3691a
:020000040000fa
:2057a0000b43d3610d4b5861986041331878a0431870d3690a481943d1618022094b92004b
:020000040000fa
:2057c0005a619a6049331a780749a2431a70074afcf764fb10bdc046000400400044004108
:020000040000fa
:2057e0005816002080440041dd520000fc9e0000f7b5fff78bfb0023764c2370fff7d2f9ec
:020000040000fa
:205800000028fbd020780528f8d800f00bfc03f7304af773704a0421535e002b10d012215d
:020000040000fa
:20582000515e00290cd06d4a0020105e6c4a0025525f92109d1aa84202db8918884202dd79
:020000040000fa
:205840000923237009e0617800290ad19b18984207da02232370fef7ddfc2000fcf7c8fbf9
:020000040000fa
:20586000cce701232370a378002be9d1f5e75d4b1b68142b09dca0225b4b52001b68934281
:020000040000fa
:20588000bcdd5a4b1b68502bb8dd032320002370fcf7aefb564b1b686360a36000f082fa6c
:020000040000fa
:2058a000ace7514b1968524b0a001b68283204db626850489a1a8242a0dd05222270fa22a9
:020000040000fa
:2058c00092009b18e3604c4b200000229b5ee16123826382494b00229b5ea382e382484bd6
:020000040000fa
:2058e00000229b5e23836383fcf782fb238c0133238483e7404f0022bb5e1221625e9a4204
:020000040000fa
:2059000000dd63821021625e9a4200da23823b4e0022b35e1621625e9a4200dde382142173
:020000040000fa
:20592000625e9a4200daa382354b019300229b5e1a21625e9a4200dd63831821625e9a422e
:020000040000fa
:2059400000da23832a4de2682b689b1a31d41023e25e1221635ed21a8b235b009a4216dc8f
:020000040000fa
:205960001421625e1620215e521a9a420fdc1821625e1a20215e521a9a4208dc0f3b200002
:020000040000fa
:20598000ff3b2370fcf734fb0020fcf757fefa222b6892009b18e3600022bb5e23826382b4
:020000040000fa
:2059a0000022b35ea382e382019b00229b5e238363830d4be2691b689b1a5b119b18a0222b
:020000040000fa
:2059c000e3615200934200dc18e72b686360032337e7c046801800201c0300205415002061
:020000040000fa
:2059e000721500202c160020181600201c1600206c150020dc050000141500201c150020e2
:020000040000fa
:205a000024150020002210b5034b04491a700448044afcf743fa10bd80180020f15700008a
:020000040000fa
:205a2000a818002037a0000010b5fff7f5fc10bd10b5fbf781fd0a48fbf754fe002809d06a
:020000040000fa
:205a4000fbf77afd074b18783038c0b2092802d8fff70cfe10bd0222034b1a70fae7c04666
:020000040000fa
:205a6000fe9c00005f0000206000002010b50248fbf76cfe10bdc04658a50000034b1a6882
:020000040000fa
:205a8000034b52429b69584310407047d00f00201c03002010b5054b01301b68ff308000c8
:020000040000fa
:205aa00004220349c018fcf7f1fb10bdd40f0020d01a002010b5fdf7d7fe10bd55230849bf
:020000040000fa
:205ac00010b50b708b8801304b80064bff301b6880000422c018fcf749fcfdf7c5fe10bd3a
:020000040000fa
:205ae000d01a0020d40f002000235a2006495a5c01338018c0b2202bf9d14042c0b243422b
:020000040000fa
:205b00005841c0b27047c046d81a002070b50400fff7b4fffcf758fc002398420ad10b4b64
:020000040000fa
:205b2000202298690a4960430a4dfcf7affb002802d1e343180070bdfff7d6ff0028f8d017
:020000040000fa
:205b40002b7a462bf5d1ab89f4e7c0461c030020d81a0020d01a002070b500250c4b0d4a01
:020000040000fa
:205b60001868916900f07cfa2c00c6b2b44201d1280070bd2000fff7c9ff002804dd002d70
:020000040000fa
:205b800001d0854200da85b20134e4b2eee7c046d40f00201c030020f7b5fbf7cdfc2a4b98
:020000040000fa
:205ba00001251b782d2b02d1fbf76cfc023dfbf76ffd264b1c78002c0ad1254b4543186886
:020000040000fa
:205bc000244b9969002d11d12900234801f056fcf7bd2000fff772ff22e00134e4b2802cba
:020000040000fa
:205be00013d1fbf705ff1be01c4827e000f038fa2600c3b20193019b9e42e5d03000fff7bd
:020000040000fa
:205c000085ff771cffb2a8421bd12000fff742ff134b1a78552adcd15a889b889a42dcd1e5
:020000040000fa
:205c20003000fff72bff04003800fff727ff011b2000fcf7fdfb0028d6d00a4801f036fc52
:020000040000fa
:205c4000c6e73e00d7e7c0465f00002060000020d40f00201c03002058a0000074a0000048
:020000040000fa
:205c6000d01a00206da00000f7b5194b194f1868b96900f0f5f90025c3b20193019becb2ad
:020000040000fa
:205c8000a34203d8144801f011fcf7bd2000fff73dff01340600e0b2002e0dd0fff7eefe2a
:020000040000fa
:205ca0003100ba69030a6a430c48120a9bb292b201f0e4fb0135e1e7fff7e0feba69030a03
:020000040000fa
:205cc0006a43120a290006489bb292b2f0e7c046d40f00201c030020baa0000084a0000056
:020000040000fa
:205ce000a0a00000f7b5fcf73ff8fff735ff2a4ca080fdf7bafda388002b04d001339bb278
:020000040000fa
:205d0000002b3fd0a3808025013dedb2ff2d0ed02800fff7bffe2378552bf5d1a3886288c9
:020000040000fa
:205d2000002b03d0d31a1bb2002b05dda280a388002b01d10133a3800023184fa362e36229
:020000040000fa
:205d4000174bb969186800f08bf90100c3b2a088c9b20138019300f0f3faceb2350028002b
:020000040000fa
:205d6000fff7d4fe0200681cc0b2002a0cd1bb696b43e362fff782fea062201dfcf738f96c
:020000040000fa
:205d80000020febd0123bde7019b9842ad410540b542e4d1f1e7c046d01a00201c030020e4
:020000040000fa
:205da000d40f0020012310b502480370fcf720f910bdc046001b0020002210b5024b1a7062
:020000040000fa
:205dc000fdf752fd10bdc046001b00200023010070b502000500437020315a3310780132d6
:020000040000fa
:205de0001b18dbb28a42f9d1134c5b426b701348fcf7befce26aa36a9a420dd323003033d3
:020000040000fa
:205e00001b78002b06d1002520003130fcf7cefc280070bdfff7d0ff230030331b78002b2c
:020000040000fa
:205e2000f1d029002022e06afcf7a0fae36a01252033e362e8e7c046d01a0020011b002039
:020000040000fa
:205e400010b5fff789fe431e9841c0b210bd044bd86a9b6ac01a43425841c0b27047c046ca
:020000040000fa
:205e6000d01a0020002210b5064b07481a70074b09321a70fbf76afc054a06490648fcf7b9
:020000040000fa
:205e80000df810bd001b0020cca50000021b0020bfa000009d5e0000081b0020f7b5fdf70a
:020000040000fa
:205ea000e4fcfff71fff4e4d2b78002b58d046234c4c23704c4b20001b6863804b4b1b8873
:020000040000fa
:205ec000e3804b4b1b8823814a4b1b8863814a4b1b88a381494b1b682361494b1b68636194
:020000040000fa
:205ee000484b1b68a361484b1b88a380fff76eff1f22464b464e01931b7801331340454a29
:020000040000fa
:205f000033705b019b5800220093434b1a70019b32781b789a4227d1404b3f4f1b783a78b7
:020000040000fa
:205f20009a4211d03b7053232370fcf735fb3b786080a38000232000e380fff747ff3b7882
:020000040000fa
:205f4000082b01d1fff738fffff7b4fd0a20fcf7c5f82b78002bdad12800fcf721f8f8e702
:020000040000fa
:205f60002800fcf71df89ee72a4b5201d75800996780791a2ed49b1841219a8a2000524273
:020000040000fa
:205f8000a2805a8a21705242e280da8a22815a8b524262811a8b5242a2819a8be281da89ca
:020000040000fa
:205fa00022829a8962821a8a5242a2821a89e2829a88db886283a383194b1b88e383fff7e0
:020000040000fa
:205fc00005ff3a00144b0a321b780092052b01d87b1c00931f22337801331340337096e7fd
:020000040000fa
:205fe000001b0020d81a00206c1500205415002056150020581500205a15002064150020ea
:020000040000fa
:206000005c15002060150020d41a00203c070020341d002040070020021b0020801800201c
:020000040000fa
:206020005416002002b4714649084900095649008e4402bc7047c04602b4714649084900d3
:020000040000fa
:20604000095c49008e4402bc7047c04603b47146490840004900095e49008e4403bc704705
:020000040000fa
:20606000002243088b4274d303098b425fd3030a8b4244d3030b8b4228d3030c8b420dd311
:020000040000fa
:20608000ff22090212ba030c8b4202d31212090265d0030b8b4219d300e0090ac30b8b429e
:020000040000fa
:2060a00001d3cb03c01a5241830b8b4201d38b03c01a5241430b8b4201d34b03c01a5241fd
:020000040000fa
:2060c000030b8b4201d30b03c01a5241c30a8b4201d3cb02c01a5241830a8b4201d38b0233
:020000040000fa
:2060e000c01a5241430a8b4201d34b02c01a5241030a8b4201d30b02c01a5241cdd2c309f8
:020000040000fa
:206100008b4201d3cb01c01a524183098b4201d38b01c01a524143098b4201d34b01c01a6c
:020000040000fa
:20612000524103098b4201d30b01c01a5241c3088b4201d3cb00c01a524183088b4201d3d6
:020000040000fa
:206140008b00c01a524143088b4201d34b00c01a5241411a00d20146524110467047ffe7a9
:020000040000fa
:2061600001b5002000f0f0f802bdc0460029f7d076e7704703460b437fd4002243088b4284
:020000040000fa
:2061800074d303098b425fd3030a8b4244d3030b8b4228d3030c8b420dd3ff22090212ba32
:020000040000fa
:2061a000030c8b4202d31212090265d0030b8b4219d300e0090ac30b8b4201d3cb03c01af9
:020000040000fa
:2061c0005241830b8b4201d38b03c01a5241430b8b4201d34b03c01a5241030b8b4201d3a9
:020000040000fa
:2061e0000b03c01a5241c30a8b4201d3cb02c01a5241830a8b4201d38b02c01a5241430a07
:020000040000fa
:206200008b4201d34b02c01a5241030a8b4201d30b02c01a5241cdd2c3098b4201d3cb0123
:020000040000fa
:20622000c01a524183098b4201d38b01c01a524143098b4201d34b01c01a524103098b424c
:020000040000fa
:2062400001d30b01c01a5241c3088b4201d3cb00c01a524183088b4201d38b00c01a524129
:020000040000fa
:2062600043088b4201d34b00c01a5241411a00d201465241104670475de0ca0f00d04942f5
:020000040000fa
:20628000031000d34042534000229c4603098b422dd3030a8b4212d3fc22890112ba030ae6
:020000040000fa
:2062a0008b420cd3890192118b4208d3890192118b4204d389013ad0921100e08909c30917
:020000040000fa
:2062c0008b4201d3cb01c01a524183098b4201d38b01c01a524143098b4201d34b01c01aab
:020000040000fa
:2062e000524103098b4201d30b01c01a5241c3088b4201d3cb00c01a524183088b4201d315
:020000040000fa
:206300008b00c01a5241d9d243088b4201d34b00c01a5241411a00d20146634652415b101b
:020000040000fa
:20632000104601d34042002b00d54942704763465b1000d3404201b5002000f005f802bd84
:020000040000fa
:206340000029f8d016e770477047c046844608006146ffe71fb500f071fc002801d400212d
:020000040000fa
:20636000c8421fbd10b500f0f7fb4042013010bd10b500f063fc002801db002010bd0120ea
:020000040000fa
:2063800010bdc04610b500f059fc002801dd002010bd012010bdc04610b500f005fc00285b
:020000040000fa
:2063a00001dc002010bd012010bdc04610b500f0fbfb002801da002010bd012010bdc04690
:020000040000fa
:2063c000002b11d1002a0fd1002900d1002802d00021c943080007b4024802a140180290eb
:020000040000fa
:2063e00003bdc04665ffffff03b4684601b5029800f034f8019b9e4602b00cbc7047c046ed
:020000040000fa
:20640000f0b5ce469946030c9c46130447461b0c1d000e0061460404240c80b50700100cc6
:020000040000fa
:206420004b436543414360432c0cc01824188c46a34203d980235b029846c44449467943ef
:020000040000fa
:206440005643230c2d042d0c8919634424046019c918c0bcb946b046f0bdc046f0b55746d9
:020000040000fa
:206460004e464546de46e0b504000d009246994683b08b4230d82dd04946504600f0b4ffaf
:020000040000fa
:2064800029000600200000f0afff331a9846203b34d49b4653465a46934042461f00534654
:020000040000fa
:2064a00093401e00af423bd8af4200d179e05b46a41bbd41002b00da76e00022002300923c
:020000040000fa
:2064c000019301235a4693400193012342469340009329e08242cfd900220023009201930b
:020000040000fa
:2064e0000c9b002b01d01c605d600098019903b0f0bcbb46b246a946a046f0bd42469b464b
:020000040000fa
:2065000020239b1a5246da40414613004a468a40170042461f43534693401e00af42c3d9c5
:020000040000fa
:2065200000220023009201934346002bd8d0fb0772081a4346467b080ee0ab4201d1a2421b
:020000040000fa
:206540000cd8a41a9d41012024196d410021013e24184d41002e06d0ab42eed9013e241951
:020000040000fa
:206560006d41002ef8d1009801995b4600196941002b24db2b005a464446d3402a00e24002
:020000040000fa
:206580001c005b461500002b2adb26009e40330026004746be403200801a99410090019149
:020000040000fa
:2065a0009ee7a342bcd882e74246202300219b1a0022009101920122da40019285e74246c9
:020000040000fa
:2065c00020239b1a2a0046469a402300f340444613432a00e2401c005b461500002bd4da06
:020000040000fa
:2065e00042462f002023260097409b1ade403b003343cde7f0b5c64643025b0a9c461f0010
:020000040000fa
:20660000de004b025a0a450090464a002d0e120ec40f00b5c90f9b09a81a8c4221d000287e
:020000040000fa
:206620000ddd002a2dd1002b00d195e0421e012800d131e1ff2800d194e0100027e00028c0
:020000040000fa
:2066400062d0501b002d00d0e1e0002e00d181e0441e012800d142e1ff2800d119e12000ee
:020000040000fa
:20666000dae0002800dc9ce0002a69d0ff2d00d178e08022d20413431b2800dc7de00136a7
:020000040000fa
:206680002ae0ff2d00d16de08022d204134301221b2807dc2021091a1a008b40c240591ecd
:020000040000fa
:2066a0008b411a43b61a730100d477e0b601b709380000f07bfe05388740854200dd82e020
:020000040000fa
:2066c00020223b00401b0130121a3e009340c6405a1e934100251e43730704d00f233340a9
:020000040000fa
:2066e000042b00d00436730137d5681cfe2d52d08e4bc0b233409b015f0ac0053843e40722
:020000040000fa
:20670000204380bcb846f0bdfe206a1c104274d1002d00d0aae0002e00d1dae00020002b69
:020000040000fa
:20672000ebd08022f71ad204174200d1ece09b1b134200d1f2e07d4a0c0013400130dae759
:020000040000fa
:20674000002b09d0421e012800d196e0ff2809d0100091e70c001e000500f3089c46ff2da5
:020000040000fa
:2067600000d091e06346002b15d080276346ff031f437f02ff207f0abfe72021091a1a001e
:020000040000fa
:206780008b40c240591e8b411343f618730105d50135ff2d54d1ff200027aee773079dd1ed
:020000040000fa
:2067a000dbe7002813d0501b002d50d1002ed2d0411e012840d0ff286cd008001b286eddf2
:020000040000fa
:2067c00015005e1c88e7594e2d1a3e4084e7fe216a1c114241d1002d6cd1002e00d190e001
:020000040000fa
:2067e0000020002b00d188e7f318df087f027f0a5b0100d481e701207fe7f71a7a0132d461
:020000040000fa
:20680000002f00d054e700240020002775e7ff2a3fd08024e404264301241b2808dc3500c9
:020000040000fa
:206820001f34241aa640c540741ea6412c0034431e1b15000c0036e7f6180235730120d59b
:020000040000fa
:2068400001233b4a3340760816401e4344e7ff2a20d08021c9040e43b0e7ff2a9bd0f618ab
:020000040000fa
:206860001500760838e70c009f1b21e7002e3ad1002b4ed0c4460c0077e7f61802257301f9
:020000040000fa
:20688000ded4f3089c46012563465f027f0ae8b233e70c00c44665e70125f61a03e7310049
:020000040000fa
:2068a0002025c140281a8640701e86410e431500f6186be7002eedd0002b00d155e78023a9
:020000040000fa
:2068c000db039c4500d250e7984500d34de7c4464be7002b97d00c00474600200de70c0085
:020000040000fa
:2068e0009e1b0135dfe6002b00d13ee78023db039c4500d239e7984500d336e70c00c4468c
:020000040000fa
:2069000033e747460020f8e6002f0bd0bf017f0af3e680270024ff20ff03eee69b010c003e
:020000040000fa
:206920005f0aeae600240027e7e6c046fffffffbffffff7df0b546464f46d6464502c0b5f0
:020000040000fa
:20694000c30f470098460e1c6d0a3f0e57d0ff2f21d08023ed00db041d43002399469a465b
:020000040000fa
:206960007f3f74027300640a1b0ef60f002b20d0ff2b4cd080220020e400d20414437f3be6
:020000040000fa
:206980004246ff1a4b4672400f2b00d9ace06f499b00cb589f46002d5bd108239946063b75
:020000040000fa
:2069a00074029a467300ff27640a1b0ef60f002bded1002c30d101234246494672401943fc
:020000040000fa
:2069c0000e2904d86248890041588f464246ff200024c0052043d2071043e0bcba46b14651
:020000040000fa
:2069e000a846f0bd5346022bf0d0032b00d1a3e042462c00012b35d100200024e9e7002dcd
:020000040000fa
:206a00001bd104239946033b00279a46a9e7002c0cd10223ff3fcfe7200000f0c7fc431f58
:020000040000fa
:206a20009c4076235b421b1a0020a9e703234a461a4391460320fc33a2e7280000f0b6fcd0
:020000040000fa
:206a40007627431f9d4000237f4299469a463f1a87e70c239946093bff279a4681e7032805
:020000040000fa
:206a60006cd0320038007f30002825dd630704d00f232340042b00d00434230103d5380059
:020000040000fa
:206a8000344b80301c40fe28a1dca401640ac0b29fe780240022ff20e4039ae78023db03ef
:020000040000fa
:206aa0001d4201d01c424bd08024e4032c4364024246ff20640a8ce701231b1a1b2b9bdc2f
:020000040000fa
:206ac00021009e37d940bc400b00611e8c412343590704d00f211940042900d004335901a3
:020000040000fa
:206ae00026d50120002474e76d016001854213d21b230024013f0126290064006d00002994
:020000040000fa
:206b000001dba84201d82d1a3443013b002bf3d16b1e9d412c43a5e71a2301242d1aeae711
:020000040000fa
:206b2000981e43425841404232000024c0b250e79b0100205c0a4ce746462c008023db0372
:020000040000fa
:206b40001c4364023200ff20640a42e710a6000050a60000fffffff770b542004e024c00e5
:020000040000fa
:206b600045026d0a120ec30f760a240ec90fff2a10d0ff2c0cd00120a2420ad1b54208d11b
:020000040000fa
:206b80008b420fd0002a04d12800431e984100e0012070bd0120ff2cfbd13543f9d14b40d5
:020000040000fa
:206ba0001800f6e70020f4e730b5420044024d02c30f4800640a120e6d0a000ec90fff2afb
:020000040000fa
:206bc00017d0ff280ad0002a1bd100280ad1002d24d0002c2ed14800013830bd002d26d1d6
:020000040000fa
:206be000002a01d1002cf6d08b4206d158000138f3e7002c1bd1ff2813d001205b4218435d
:020000040000fa
:206c0000ebe70028f9d08b42f7d18242f5dceddbac42f2d80020ac42dfd2e7e7002cdcd0a2
:020000040000fa
:206c2000ebe7002d03d18b42e7d10020d5e702204042d2e78b42ebd0dfe7c04630b5420048
:020000040000fa
:206c400044024d02c30f4800640a120e6d0a000ec90fff2a18d0ff280dd0002a1cd1002846
:020000040000fa
:206c60000dd1002d27d0002c0bd08b421bd001205b4218430fe0002d0cd1002a1ed1002cfc
:020000040000fa
:206c80001cd14800013806e0002c03d1ff28eed1002d16d0022030bd0028e8d08b42e6d134
:020000040000fa
:206ca0008242e4dc04dbac42e1d80020ac42f2d258000138efe7002cedd0d8e78b42d6d175
:020000040000fa
:206cc000f6e700208b42e6d0d1e7c046f0b54f464646d6464502c0b546000f1c6d0a360eac
:020000040000fa
:206ce000c40f002e00d1c3e0ff2e77d08023ed00db041d43002399469a467f3e7b025b0a5b
:020000040000fa
:206d000098467b001b0eff0f002b77d0ff2b00d194e042468021d200c904114388460021f7
:020000040000fa
:206d20007f3bf6184b46721c0a2b73dc4b467c40022b00dca7e0484601238340a620c00010
:020000040000fa
:206d4000034267d190208000034200d0ece0b938ff38184200d0dae041460904090c434667
:020000040000fa
:206d60000f00280c2d041b0c2d0c6f4341435d4358436d183b0c5b19994203d980214902eb
:020000040000fa
:206d80008c4660443f0419043f0cc9198d016f1ebd411b0c890e1b180d439b011d431b017e
:020000040000fa
:206da00000d4c6e0012369081d400d4310007f30002800dc94e06b0704d00f232b40042bce
:020000040000fa
:206dc00000d004352b0103d5803210005e4b1d40fe2855dcab015b0ac0b226e0002d00d001
:020000040000fa
:206de00078e008239946063b9a467b025b0a98467b00ff261b0eff0f002b87d14346002b42
:020000040000fa
:206e000056d14a4601331a4391464b460121721c0a2b8bdd5346022b32d0032b00d17ce052
:020000040000fa
:206e20005346012bc2d100200023c0051843e4072043e0bcba46b146a846f0bd3300424660
:020000040000fa
:206e4000ff33002a3fd0032249461143721c8946ff320a2973dd0f295dd18023db031d4268
:020000040000fa
:206e60005bd042461a4258d13c00ff201343dce7002d11d104239946033b00269a463de7e9
:020000040000fa
:206e8000ff200023d1e7013b012b00d964e70229f6d045468a46c3e7280000f087fa762641
:020000040000fa
:206ea000431f9d400023764299469a46361a25e7404600f07bfa4246431f9a40361a9046c8
:020000040000fa
:206ec0000021763e2ee749460232114389461e00022127e70c239946093bff269a460de748
:020000040000fa
:206ee00001231b1a1b2b9edc9e3229009540d9406a1e95410d436b0704d00f232b40042bd2
:020000040000fa
:206f000000d004356b0116d5012000238de73c0045468a467ee73c0045468023db032b43a7
:020000040000fa
:206f20005b02ff205b0a80e780230024ff20db037be732003ae7ab0100205b0a75e71e00e5
:020000040000fa
:206f400003217c40f7e6c046fffffff7f0b546464f46d64643025b0ac0b59c461f00de009a
:020000040000fa
:206f60004b025a0a904645004a002d0ec40f120ec90f9b09ff2a26d001204140a81a8c4200
:020000040000fa
:206f800010d0002800dc8ae1002a48d1002b00d1aee0421e012800d13fe1ff2800d1ade0d6
:020000040000fa
:206fa000100041e0002800dc86e1002a00d182e0ff2d00d1a2e08022d20413431b2800dc6c
:020000040000fa
:206fc00083e0013654e02800ff388246002b69d1012041408c4200d1d8e05046002800d1cf
:020000040000fa
:206fe0009ae00c00002d00d07de0ff20002e00d17ce0471e012800d12ce10c00ff2800d1c7
:020000040000fa
:2070000009e101211b2f07dc2020c01b31008640f940701e8641314315005e1a10e0ff2d7a
:020000040000fa
:207020006cd08022d204134301221b2807dc2021091a1a008b40c240591e8b411a43b61a42
:020000040000fa
:20704000730166d5b601b709380000f0aff905388740854200dd7ae020223b00401b01302f
:020000040000fa
:20706000121a3e009340c6405a1e934100251e43730704d00f233340042b00d0043673015b
:020000040000fa
:2070800037d5681cfe2d2ed0914bc0b233409b015f0ac0053843e4072043e0bcba46b14650
:020000040000fa
:2070a000a846f0bd8c4260d0002835d0002d9cd00c00c44622e0002b1ad0421e012800d1ea
:020000040000fa
:2070c0009de0ff281ad0100078e72021091a1a008b40c240591e8b411343f618730118d560
:020000040000fa
:2070e0000135ff2d6ad1ff200027d2e70c001e000500f3089c46ff2d00d087e06346002bb1
:020000040000fa
:20710000f1d080276346ff031f437f02ff207f0abfe77307aed1ece7fe206a1c10421ad17e
:020000040000fa
:20712000002d63d1002e00d198e00020002bb0d08022f71ad204174200d1a8e001249b1b96
:020000040000fa
:207140000c401342a3d0624a013013409fe7604e2d1a3e408ce7f71a7a0143d4002f00d0dd
:020000040000fa
:2071600072e700240020002793e7002811d0002d51d1ff20002ebad0411e01283fd0ff28e4
:020000040000fa
:2071800049d01b294cdd15005e1c71e7514600291bd1fe216a1c11421ed1002d4bd1002e78
:020000040000fa
:2071a00072d00020002b00d173e7f318df087f027f0a5b0100d46ce701206ae70123454a73
:020000040000fa
:2071c0003340760816401e4352e7002dd1d08ae7fe216a1c0a42e2d0ff2a84d0f61815004c
:020000040000fa
:2071e000760845e701249f1b0c402de7002e3cd1002b45d180270024ff20ff0349e7f61800
:020000040000fa
:2072000002257301dad4f3089c46012563465f027f0ae8b23de7c44670e70125f61a0fe744
:020000040000fa
:2072200030002025c840691a8e40711e8e4106431500f61852e7002eedd0002b00d160e74f
:020000040000fa
:207240008023db039c4500d25be7984500d358e7c44656e70c0001259e1bf1e6002b80d045
:020000040000fa
:207260000124474600200c4013e7002b00d148e78023db039c4500d243e7984500d340e796
:020000040000fa
:207280000124c4460c403ce74746002001e7002f02d0bf017f0afce600240027f9e600283d
:020000040000fa
:2072a00000d139e7571b3800002d00d19ee68020c0040c000643a4e6002889d0511b002d54
:020000040000fa
:2072c00001d1080056e78020c004064359e7c046fffffffbffffff7d41024200c30f490a88
:020000040000fa
:2072e0000020120e7e2a03dd9d2a02dd094a98187047802000040143952a07dc9620821a8a
:020000040000fa
:20730000d1404842002bf3d10800f1e7963a9140f7e7c046ffffff7f70b5002813d0c317f8
:020000040000fa
:20732000c5185d40c40f280000f040f89e2301001b1a962b0fdc082831d008398d406d025f
:020000040000fa
:207340006d0ad8b202e0002400200025c0052843e407204370bd992b15dc421f95402a0021
:020000040000fa
:20736000150011480540560709d00f263240042a05d004356a0102d59f2305405b1aad01d5
:020000040000fa
:207380006d0ad8b2e2e70522121a2800d0400a001b3295402a00551eaa410243e0e76d0269
:020000040000fa
:2073a00096206d0ad2e7c046fffffffb1c2101231b04984201d3000c10391b0a984201d393
:020000040000fa
:2073c000000a08391b09984201d30009043902a2105c40187047c046040302020101010116
:020000040000fa
:2073e000000000000000000010b5002903d1fff7ddff203002e00800fff7d8ff10bdc0461f
:020000040000fa
:2074000002780b78002a03d0013001319a42f7d0d01a7047002310b59a4200d110bdcc5c41
:020000040000fa
:20742000c4540133f8e710b5884202d98b18984208d300239a4207d0cc5cc4540133f9e735
:020000040000fa
:207440008b5c8354013afbd210bd03008218934200d1704719700133f9e70023c25c01338d
:020000040000fa
:20746000002afbd1581e70470023c26810b59a4201d090470300180010bd00000fb407b5ec
:020000040000fa
:20748000054b04aa02ca1868019200f0f1f803b008bc04b01847c0461ca3000010b5024bd5
:020000040000fa
:2074a000196801f02bfd10bd1ca30000f8b50e4b04001d68ab789b0713d56e6827782900cc
:020000040000fa
:2074c000002f05d10a20b047002806db38000ae03800b04701340028f0da0423aa78134366
:020000040000fa
:2074e000ab7001204042f8bd1ca30000f7b50d003721c91ac9b201911f21040016000027d8
:020000040000fa
:207500000b400093200029003b00009afef758ffd2b2a4462b0004000d00092a02d90199d1
:020000040000fa
:207520008a18d2b23032701c32709f4203d803d1009b634500d9febd0600e3e7f0b5012593
:020000040000fa
:2075400085b0029001910392029c039bab4201dc05b0f0bd23001c0022780133002af7d0d7
:020000040000fa
:20756000252af8d11a780234252af3d00020060003000094009c1f2b27d8202149428c46d9
:020000040000fa
:2075800094446146102907d867463849f9400127394251d12e2a3dd02e2a24d8242a35d01c
:020000040000fa
:2075a0002a2a37d0002ed3d0ae42ced1202414432000019965380e68022801d9612c41d105
:020000040000fa
:2075c0000723f01d984308304be07f2be2d96c2a27d021d8682a2cd06a2a01d04c2ae1d130
:020000040000fa
:2075e000a022920023e0302149428c46944461460929ecd80a23584316336044009a01328f
:020000040000fa
:2076000000922278002ab5d1009ccbe7002e15d0a84215d00020f1e7742aefd07a2aedd0a8
:020000040000fa
:20762000c0e78022134202d0802189000b431343e4e780225200f5e70023dfe70600e9e7b2
:020000040000fa
:207640006322b3e7692a04d0301d692a07d8632a07d0301d1a0604d59b0502d5b0e7732a90
:020000040000fa
:20766000f7d1019b013518606ee7c04689280100f0b543689bb004900f91109205938378e7
:020000040000fa
:207680009b0718d50b00002713921878002800d10de1252812d001330d930499059b013795
:020000040000fa
:2076a0009847002801db00f0eafb049b9a7804231343049a937001277f42f8e05d789a1cf7
:020000040000fa
:2076c0000d92252de9d0002634000d9b039609930896099b0d931f2c19d8280020381028f3
:020000040000fa
:2076e00018d8fef7a9fc0e171712171717be1717170c17101717090001231c43b1e00223c7
:020000040000fa
:207700001c430423f9e70823f7e71023f5e77f2c00d9e5e02e2d00d1c5e000d996e0242d31
:020000040000fa
:2077200000d1c7e02a2d00d1ace0002e06d0109b32000f9813a91393fff700ff039b002b75
:020000040000fa
:2077400003da40239c430023039320231a002a430a92653a022a03d90a9a612a00d0bae2a9
:020000040000fa
:207760000722ab430e93139b073393431a001d685e684023083213920a9a2340612a00d08a
:020000040000fa
:20778000d1e0c02252011443002b01d1013b03930e9b310000932800039b14aa01f010fbf0
:020000040000fa
:2077a00003000133dbb20b930123149e0c936f3303900a9333000933122b0dd902230c93ca
:020000040000fa
:2077c00033006333c62b07d97f4a804bb21893429b415b4203330c93012214ab1b792d25c6
:020000040000fa
:2077e000134205d1023da10702d4a50815406d010c22134200d1dbe02b005a1e9341089a09
:020000040000fa
:20780000033393420edad31a099324070cd4dc1920200499059b01379847002800da44e72b
:020000040000fa
:20782000bc42f5d100230993002d07d028000499059b01379847002800da36e714ab1b79d3
:020000040000fa
:20784000634c1b0700d4634c3d00abe02a00303a092a45d80a2361060ed503994b439b18d4
:020000040000fa
:207860000393099b013309930d9b1d78002d00d02fe7099b0d9358e708994b439b180893ae
:020000040000fa
:2078800020233ae7002eecd1139a08ca13926106e6d4002b03db202214430893e1e75b42b2
:020000040000fa
:2078a0000893282329e740231c4200d125e738001bb0f0bd002e30d0109b2500139340237d
:020000040000fa
:2078c000089a1d401c4200d0039a0f9813a9fff735fe139b1a1d13921b68002dddd0bfe7c5
:020000040000fa
:2078e0006c2d0fd009d8682d14d06a2d02d04c2d00d01ae7a0239b00ffe6742db1d07a2df7
:020000040000fa
:20790000afd012e780231c4200d1f6e6802292001443f2e680235b00f5e70396039b089e27
:020000040000fa
:207920001c0008939de7002b01d1063303930a9b652b18d10021039b08005a1c80235b01e6
:020000040000fa
:20794000d2b21c43131c112a15d8dbb2019000912800310014aa00f067fcc3b20b9302239c
:020000040000fa
:20796000149e0c9326e70a9b662b06d1802301219b0103981c431123e7e76b461a7b002acf
:020000040000fa
:2079800000d10122002165230800d2b20a93d9e70e9b0499c01ac0b2059b013598470028f2
:020000040000fa
:2079a00000da82e6e31b585d0028f1d12f0028e3c0239b011c422fd1039b002b00d1aae0ad
:020000040000fa
:2079c0000b9a14ab9b180be0e7030000ce070000c7a00000c3a000000b9a013ad2b20b921b
:020000040000fa
:2079e0000b9a002a03d01a79013b302af4d0039be20600d40b9b321d00da8fe0039a9642eb
:020000040000fa
:207a000000db8be080229201144300220392b34202dd721c9b1a0393802322009b011a4075
:020000040000fa
:207a200011921c427cd0f343db17334001332a00511e8a419b18039a002a78d001329b181e
:020000040000fa
:207a400000220992089a9a4201ddd31a099309231c4207d1099bdb190893089b9f4269d131
:020000040000fa
:207a600000230993002d07d028000499059b01379847002800da18e6230511d530200499cc
:020000040000fa
:207a8000059b9847002800da0fe678200e9b0499c01ac0b2059b02379847002800da04e6a2
:020000040000fa
:207aa000230705d4099bdd19af424bd100230993119b002b71d0f343db171a0032400892f7
:020000040000fa
:207ac00032009a430a920b9b0a9a3020934203d9130014aa9b185879089b7d1c013b089348
:020000040000fa
:207ae000039b089a5b42934234dc059b049998470a9b01330a93002800dad6e5089b01339e
:020000040000fa
:207b000007d12e200499059b9847002800dacce5bd1c2f00d7e70123039351e7013b7ae71b
:020000040000fa
:207b20000523220500d4023b0c9ad3187fe7e206d20f84e720200499059b013798470028fe
:020000040000fa
:207b40008bdab2e530200499059b984701370028aadaaae5089b9e4207d114ab5a79352afe
:020000040000fa
:207b600019d802d11b79db0615d50499059b9847002800da99e5e40600d417e7089b0133b3
:020000040000fa
:207b800000d013e72e200499bd1c059b9847002800db0be789e53120e7e714aa5079312876
:020000040000fa
:207ba00003d0102113798b4313710499059b9847002800da79e5039b002b74dd2e20049962
:020000040000fa
:207bc000059b9847002800da6fe5012430250b9b28000894a34202dd14abe3185879049900
:020000040000fa
:207be000059b9847002800da5fe5039b0134a342edda089b0237fd180a9b0e9a0499981ab4
:020000040000fa
:207c0000c0b2059b9847002800da4ee5002e06db2b20002e05d114ab1b79db0601d52d2089
:020000040000fa
:207c200076420499059b9847002800da3de50c9b042b43d1fa2130008900fef79bfa3030a4
:020000040000fa
:207c40000499059bc0b203359847002800da2ce5fa2130008900fef773fb0e006421300051
:020000040000fa
:207c6000fef788fa30300499059bc0b201359847002800da19e530006421fef761fb0e0055
:020000040000fa
:207c80000a213000fef776fa30300499059bc0b201359847002800da07e530000a21fef7c2
:020000040000fa
:207ca0004ffb0e0011e07d1ce406a5d52e200499059bbd1c984700289edaf6e40c9b0235e3
:020000040000fa
:207cc000032bcbd00c9b012bdad13000303004990135c0b259e728006338122800d9b6e0dc
:020000040000fa
:207ce000fef7aaf90a4ab5b5b5b54ab5b5b5b5b5d0b1b5b51eb59000139b14ae1a1d1b6879
:020000040000fa
:207d0000139233700123039324072ad53d00039bdc19a54227d1089b039a9b1a099345e6cc
:020000040000fa
:207d2000139b1a1d13921e68002e00d1b84e0399630601d401214942300001f035f80390c6
:020000040000fa
:207d4000e2e720200499059b9847002800daace4013c039ba342f4d3089b0894df193f1b54
:020000040000fa
:207d6000d4e7089cf5e7f31b585d0499059b984701350028cdda98e4139b220637d5a205df
:020000040000fa
:207d80002ed50722073393431a00083213921a685b6806920793079b002b09da0698079949
:020000040000fa
:207da000002342428b41069207938023db001c4310232600079a9e43069b134306d164062e
:020000040000fa
:207dc00004d50a93039b002b00d182e00698079914ac0a232200fff789fb031b0a9378e057
:020000040000fa
:207de0001a1d1b6813920693db170793d3e71a1d13921b68e205f6d5a20501d55bb2f2e7d1
:020000040000fa
:207e00001bb2f0e710239c43063b8021200008408446139a0c423cd080202100800001400f
:020000040000fa
:207e2000044232d0072107328a4311000831139103ca02000a43944640d0062294432600b3
:020000040000fa
:207e400014ac2200c7e7102378251c43dde70a9b782b03d15a1b683b1343d6e72520049976
:020000040000fa
:207e6000059b9847002801dafff71ffc0499059be8b29847002801dafff717fc02370d9bcc
:020000040000fa
:207e8000fff703fc08230025bfe7101d13901068cfe7111d8020139121004000126801406b
:020000040000fa
:207ea000044201d11000c4e780262100b600314090b23442bdd06146d0b2bae71626220094
:020000040000fa
:207ec000b24316006406bbd562460a92039a002ab6d10a9c099673060cd5012332009a4339
:020000040000fa
:207ee000039b0992a34205dd1c00002d02d111239e4309961023099a1a400b92099a1a42e6
:020000040000fa
:207f000016d02b005a1e93411b195c1c099b1b0724d4099bdb0709d50a9b0393089ba34273
:020000040000fa
:207f200004dd1c1b0a9be318089c039326000fe0099a384b13405a1e9341e418e6e720206c
:020000040000fa
:207f40000499059b9847002801dafff7aefb0136089bb342f3dc3f1b3400bf190b9b002b8e
:020000040000fa
:207f600014d030200499059b9847002801dafff79cfb002d30d00237e8b20499059b984705
:020000040000fa
:207f8000002801dafff791fb3d0017e0214b099a1a42f9d013002b209b0700d40b38099b39
:020000040000fa
:207fa0005b0500d52d200137e7e730200499059b01359847002801dafff777fb039b0a9aea
:020000040000fa
:207fc000fb185b1b9a42f0db1600002e06d10a9b5d19089b1b1ba1e60137d5e714ab013ee9
:020000040000fa
:207fe000f05c0499059b98470028eedafff75dfb20200499059b01379847002801dafff74e
:020000040000fa
:2080000054fb099b5b19db1b002bf1dc37e7c046cba0000006040000f0b506000f00b619e9
:020000040000fa
:208020007f418fb00aa9140009933000536812680091390000f060fca268e36805910ca9c3
:020000040000fa
:20804000049000913000390000f056fc0a9a0b9b8018594102900391039d01200021ab42df
:020000040000fa
:2080600005d802d1029daa4201d8002000210c9a0d9b8018594102000b0006900791049854
:020000040000fa
:2080800005990c920d932268636812184b41059d012000219d4205d802d1049d954201d835
:020000040000fa
:2080a00000200021029d039ea268e3685219734180185941099b039d413b1f000122002374
:020000040000fa
:2080c0008d4205d802d1029d854201d800220023069d079e00975219734100f045fc149bbf
:020000040000fa
:2080e00018605960169b012b32d1a268e368029803996568059e801a994101220023b542c3
:020000040000fa
:2081000006d803d12468049dac4201d800220023801a9941039b01240025994205d802d18d
:020000040000fa
:20812000029b984201d8002400250c9a0d9b121bab413c00009400f017fc159b03c30c9a50
:020000040000fa
:208140000d9b02980399009700f00efc0fb0f0bd049a059b1000190012184b4102980399f1
:020000040000fa
:2081600094461d0002000b00059e8018594101220023ae4205d802d1049e664501d80022f8
:020000040000fa
:2081800000238018594104900591616801220023a94205d802d12168614501d80022002369
:020000040000fa
:2081a00004980599801a9941a268e3680c9c0d9d24196d41059e06940795039c801a994193
:020000040000fa
:2081c00001220023b44206d803d1049e029cb44201d800220023069c079d059e12196b419d
:020000040000fa
:2081e00001240025b14205d802d1049eb04201d800240025121bab41099c403c9ae7000021
:020000040000fa
:208200001fb502ab0093064a064b00f075fb039902984b07c0081843c90805b000bdc04655
:020000040000fa
:20822000cdccccccccccccccf0b5a1b00c9326ab1b780b9213930a0d0b031b0b5505ce0f1f
:020000040000fa
:2082400007006c0d0e961843002d0ed1002800d082e030230b9a53712e3b334301260b9ad2
:020000040000fa
:2082600013711060300021b0f0bdca498c4209d10823002800d104230e9a002613430b9a8d
:020000040000fa
:208280001371efe7c4496418802149031943049101239c463b0061460b4004990d93890024
:020000040000fa
:2082a000bb0f1943bb00664607910693002803d1ba4b1a4056425641002c00da7de02000f3
:020000040000fa
:2082c00000f0f4f90123032c00dc0023c31a1800099300f0f7f9099b7c301c1b04191ca995
:020000040000fa
:2082e000180000f089fa18ab019316ab380000930499230002961caafff78efe0027099ba5
:020000040000fa
:20830000049005910a97152b1bd8069807991aaba34a0093a34b00f0effa169c179d1a9bfa
:020000040000fa
:208320001b9a9b089207134305225343069a934215d10698079900f0cdf9099b98427f41ac
:020000040000fa
:20834000ffb2139b0c9e002b00d19ae00a20002101260a24002582e0934c049398e70d9bda
:020000040000fa
:20836000002b15d1069b079c01204042c1171b184c413200180021000023801a994100f07b
:020000040000fa
:20838000a9f90d9b099988425b41dbb20a93d8e70220069a079b002112184b41190010003e
:020000040000fa
:2083a00000f098f93900099b984279413b000a00a41a9d4116941795c3e7634218000a9390
:020000040000fa
:2083c000012500f079f9621c00db0025451b631909930a9b5c1b200000f074f97d382b1a8c
:020000040000fa
:2083e0001ca920000a9300f08bf918ab019316ab009338000a9b049902961caafff70cfe04
:020000040000fa
:2084000004900591012d12d80d9b002b03d101273e400a9695e701204042c117169a179bd4
:020000040000fa
:2084200012184b410127169217930023aee700270a973e2d85d82a0001204042c11701f02e
:020000040000fa
:20844000fbfa069b079a83438a4313435a425341dfb276e722002b000136fdf7d1ff059bf6
:020000040000fa
:20846000994203d8f6d1049b9842f3d9099bf618279b9e19002e00dc01260c9b9e4200dd7a
:020000040000fa
:208480001e0000250695109516981799fff7b8fe189b14901191180019991593fff7b0fe40
:020000040000fa
:2084a000119b0c0012908b4203d83fd1149b83423cd904980599fff7a3fe0a22129b1994ca
:020000040000fa
:2084c0005343159a05919b1a5a4253410a9a1a400a230a926a4255414343049a2f40d31a53
:020000040000fa
:2084e000ddb2149b04901693119b1793129b1893069b01330693c7e70f9b0a2201330f938b
:020000040000fa
:208500000023fdf77dff059b994203d8f4d1049b9842f1d90f9bb3420ddd002e03d1049b40
:020000040000fa
:20852000059a134307d001231093c2e701230a2000210f93e7e70a9b002b37d0189b1999e4
:020000040000fa
:2085400018000f93fff75cfe0a2343430f9a0400119193422ad116981799fff751fe0f90fd
:020000040000fa
:20856000129104980599fff74bfe0a236a4255414343049a2f40d31addb20f9b1894169362
:020000040000fa
:20858000129b04901793119b05911993069b01330693d3e7ff070000cbfbfffffe0700000b
:020000040000fa
:2085a000cdccccccccccccccccfbffff002f06d0052d04d10123049a13400433ddb2069b0d
:020000040000fa
:2085c000099f9c46109b6744002b0ed1189b049a93420ad1199b059a934206d10d9b0124e4
:020000040000fa
:2085e000002b06d10a9b002b03d00424ac42a441644200230498059922008018594101255e
:020000040000fa
:20860000049005910a201900059b994203d83ad1049b984237d9002c20d0ae421eda139b51
:020000040000fa
:20862000002b0bd0279a7b19d318de43f6171e400c9b9e4200dd1e00b5420fdd0520049b3f
:020000040000fa
:20864000059c00211b184c410a22180021000023fdf7b6fe049005910137013d3400ae42a4
:020000040000fa
:2086600000dd2c0024b226000b9b3fb23f191d19013f0695069b5b1b9c420adc0b9b0e9acc
:020000040000fa
:208680001f601a71eee50a2200230135fdf7b8febae7049805990a220023fdf791fe3032bf
:020000040000fa
:2086a0002a7104900591013de4e7c046014b5843800c704741340100014b5843000d70479b
:020000040000fa
:2086c000fb2e0b00024b5843c00c01307047c0464f93120070b50024064d074a074bfdf79d
:020000040000fa
:2086e0008ffea94204d801d1884201d80134f4e7200070bd33333333cdcccccccccccccc27
:020000040000fa
:20870000f0b50d008db01a210490fdf7a9fc1a2105900498fdf72afd059b1c01334be41844
:020000040000fa
:20872000002909d1226863682a606b60a068e168a860e9600db0f0bd2d4bc9005b1808a91b
:020000040000fa
:208740001e685f68a268e36830000091390000f0d3f82268636803910aa9029000913000d3
:020000040000fa
:20876000390000f0c9f80a9a0b9b029e039fb6185f4106900791bb4202d809d1b24207d962
:020000040000fa
:20878000089a099b0120002112184b41089209930498fff797ff04001a20059b5843fff7ce
:020000040000fa
:2087a00091ff241a32003b0006980799009400f0dbf81e22049b0290039118090d498000ed
:020000040000fa
:2087c00041585b001a40d140032001400a0002980399002312184b4130002a606b60089a96
:020000040000fa
:2087e000099b3900009400f0bff8a1e708a8000038a7000090a60000f0b58db00390069108
:020000040000fa
:2088000019301a21fdf72cfc1a244443039b374d0001e21a45199c420bd12a686b680699b8
:020000040000fa
:208820000a604b60a868e968069b9860d9600db0f0bd2f4bd2009b1808a91e685f68aa6877
:020000040000fa
:20884000eb6830000091390000f056f82a686b680490059101204042c11712184b410aa91a
:020000040000fa
:2088600030000091390000f047f80a9a0b9b049e059fb6185f4105000791bb4202d809d183
:020000040000fa
:20888000b24207d9089a099b0120002112184b41089209932000fff715ff04000398fff7d1
:020000040000fa
:2088a00011ff241a32003b0028000799009400f05bf8039a0f4b1509ad005a191e25039b48
:020000040000fa
:2088c0005b002b40556ddd4003231d4000236a1c12184b41069930000a604b60089a099be7
:020000040000fa
:2088e0003900009400f040f89ee7c046d8a8000038a7000090a60000f0b5002487b00d0056
:020000040000fa
:2089000004932100230000920290fdf779fd009a230005900e0028002100fdf771fd2700bc
:020000040000fa
:2089200036184f41029a23002100049800960197fdf766fd2300009a270080185941049aa4
:020000040000fa
:208940000290039128002100fdf75afd019e230080197941039a801859410c9b18605960a1
:020000040000fa
:208960000598029907b0f0bdf8b50700100040220e001900069bd21a01f05ef8069a050095
:020000040000fa
:208980000c003800310001f03df828432143f8bdff214200f8b552080300041cc9058a4292
:020000040000fa
:2089a00010d3002807da00f0dbf9002803d0201c00f0f2f903e0211c201cfdf71bfe041c6c
:020000040000fa
:2089c000201cf8bd002afbd00028f0db02000a40084229d0c11580220c005b025b0a1204d3
:020000040000fa
:2089e0007f3c1a43c90700d452000023802019251f006410520040043e181100964202dc22
:020000040000fa
:208a00003718911b1b18013d4a004008002df3d1002902d0012201339343fc225b1092051f
:020000040000fa
:208a20009b18e405e418cbe7802000045b00110001320342fad04942cde70000fe21f8b58f
:020000040000fa
:208a40004300051c5b0889058b4207d10020002d08dc9a499a48fdf7cdfd03e08b4202d9dd
:020000040000fa
:208a600000f09af9f8bdfc2189058b425ad28c229205934202d893499348ece7011cfef78a
:020000040000fa
:208a800025f99249041cfef721f99149fdf7b2fd211cfef71bf98f49fef758fa211cfef79a
:020000040000fa
:208aa00015f98d49fdf7a6fd211cfef70ff98b49fef74cfa211cfef709f98949fdf79afd61
:020000040000fa
:208ac000211cfef703f98749061c201cfef7fef88549fef73bfa211cfef7f8f88349fdf775
:020000040000fa
:208ae00089fd211cfef7f2f88149fef72ffa211cfef7ecf8fe218905fdf77cfd011c301c53
:020000040000fa
:208b0000fdf718ff291cfef7e1f8011c6d48fef71dfa011c281cfef719fa011c6a48fef72c
:020000040000fa
:208b200015fa9fe700285bdafe218905fdf762fdfc218905fef7caf8041cfff729ff6349f7
:020000040000fa
:208b4000051c201cfef7c2f86149fdf753fd211cfef7bcf85f49fef7f9f9211cfef7b6f8c6
:020000040000fa
:208b60005d49fdf747fd211cfef7b0f85b49fef7edf9211cfef7aaf85949fdf73bfd211cdf
:020000040000fa
:208b8000fef7a4f85749061c201cfef79ff85649fef7dcf9211cfef799f85449fdf72afdd6
:020000040000fa
:208ba000211cfef793f85249fef7d0f9211cfef78df8fe218905fdf71dfd011c301cfdf7d0
:020000040000fa
:208bc000b9fe291cfef782f83e49fef7bff9291cfdf710fd011cfdf70dfd011c38489ee773
:020000040000fa
:208be000011cfe208005fef7b1f9fc218905fef76df8041cfff7ccfe3449061c050b201c46
:020000040000fa
:208c0000fef764f83249fdf7f5fc211cfef75ef83049fef79bf9211cfef758f82e49fdf72c
:020000040000fa
:208c2000e9fc211cfef752f82c49fef78ff9211cfef74cf82a49fdf7ddfc211cfef746f8bb
:020000040000fa
:208c40002849071c201cfef741f82749fef77ef9211cfef73bf82549fdf7ccfc211cfef779
:020000040000fa
:208c600035f82349fef772f9211cfef72ff8fe218905fdf7bffc011c381cfdf75bfe311c3b
:020000040000fa
:208c8000fef724f82d03071c291c281cfef71ef8011c201cfef75af9291c041c301cfdf796
:020000040000fa
:208ca000a9fc011c201cfdf745fe011c381cfdf7a1fc291cfdf79efc011ccce668212234fc
:020000040000fa
:208cc000da0f49406821a233da0fc93f08ef1138047f4f3a4611243da80a4e3e90b0a63e6d
:020000040000fa
:208ce000abaa2a3e2ec69d3d6133303f2d57014039d1194007b5194a43005b08934204d848
:020000040000fa
:208d00000022002100f08af905e0ff22d205934202d300f041f80ebd694600f0f1f9032373
:020000040000fa
:208d20001840012807d002280ad0002811d1012201990098e6e70199009800f0f3f8eae7cd
:020000040000fa
:208d400001220199009800f069f980231b06c018e1e70199009800f0e5f8f6e7d80f493fbd
:020000040000fa
:208d600043005a080220002b0fd0fe21074bc905d31800188b4208d30549531e01388b4273
:020000040000fa
:208d800003d9044bd018434258417047000080fffeff7f000000808010b5fff7e1ff01480c
:020000040000fa
:208da00010bdc0460000c07f030041188b4202d01a78002a01d1181a70470133f6e700001e
:020000040000fa
:208dc000f0b589b01c000eab1b78150007934b000a035b0d170b1a00024306003a4364d1a5
:020000040000fa
:208de000302303926b71cb0f02932b71002c66db0d230c2c65dc1b1b9b005a1e0120002103
:020000040000fa
:208e0000069300f019fe01910090009a019b1000190012184b4100215042994104900591c4
:020000040000fa
:208e200001204042c117801859410b000200019932403b408b420adc02d1009b9a4206d816
:020000040000fa
:208e400030003900069a00f0e9fdc0070ad5009a019bb6185f4180235b039f4202db6b7946
:020000040000fa
:208e600001336b71049a059b32403b4016001f00802203990d23d200914224d06a1d94461a
:020000040000fa
:208e800057220799521a02920f223907300932403e11009601430e00009f002a1fd19c42cf
:020000040000fa
:208ea00021da013b002befd114e03122002b01d1302201236a71104a9b18039393e70024ba
:020000040000fa
:208ec000d6e71c00d4e704233e4300d00823029a13432b712000039b2b6009b0f0bd029983
:020000040000fa
:208ee0008918092a01dc303211006246d1549c42d7da1c00d5e7c04601fcffff8b7870b5f1
:020000040000fa
:208f000004000d009b0709d54b68c0b29847e4b2002805da0423aa781343ab70012464429a
:020000040000fa
:208f2000200070bdc823f7b54400061c019164089b059c425cd3011cfdf7c8fefc218905ba
:020000040000fa
:208f4000051cfdf7c3fe2c49071c281cfdf7befe2a49fdf74ffb291cfdf7b8fe2849fdf7aa
:020000040000fa
:208f6000f5ff291cfdf7b2fe2649fdf743fb291cfdf7acfe2449fdf7e9ff291cfdf7a6fe6a
:020000040000fa
:208f80002249fdf737fb291cfdf7a0fe291cfdf79dfe0199051c301cfdf798fe011c281ca3
:020000040000fa
:208fa000fdf7d4ff1a4b051c9c4209d8011c381cfdf7ccff011cfe208005fdf7c7fffebd40
:020000040000fa
:208fc000144b9c4212d8ff231b06e418fe20211c8005fdf7bbff211c061c381cfdf7b6ff41
:020000040000fa
:208fe000291cfdf7b3ff011c301ce6e70a4cede7fe208005e3e7c0464ed747adf6740f31f0
:020000040000fa
:209000007cf29334010dd037610bb63aabaa2a3d9999993e0000483f0000903ef7b5019251
:020000040000fa
:20902000c8224300041c00915b089205934234d3011cfdf74bfe051c011c201cfdf746fe70
:020000040000fa
:209040002849061c281cfdf741fe2749fdf77eff291cfdf73bfe2549fdf7ccfa291cfdf752
:020000040000fa
:2090600035fe2349fdf772ff291cfdf72ffe2149fdf7c0fa019b071c002b10d1011c281c42
:020000040000fa
:20908000fdf724fe1c49fdf761ff311cfdf71efe011c201cfdf7aefa041c201cfebdfc217b
:020000040000fa
:2090a00000988905fdf712fe391c0190301cfdf70dfe011c0198fdf749ff291cfdf706fe26
:020000040000fa
:2090c0000099fdf743ff0d49051c301cfdf7fefd011c281cfdf73aff011c201cfdf736ffff
:020000040000fa
:2090e000dae7c046d3c92e2f342fd7321bef3836010d50398988083cabaa2a3eabaa2abee6
:020000040000fa
:20910000f0b59f4b8bb047000c00061c05907f089f4204d8002308604b6000251be0994bfd
:020000040000fa
:209120009f424cd8984d994f99490540002823ddfdf70cff061cbd4210d09649fdf706ff36
:020000040000fa
:20914000011c051c301cfdf701ff9249fdf7fefe25600125606028000bb0f0bd8e49fdf700
:020000040000fa
:20916000f5fe8e49061cfdf7f1fe011c051c301cfdf7ecfe8949e9e7fdf73cfa061cbd42cb
:020000040000fa
:209180000fd08449fdf736fa011c051c301cfdf7ddfe8049fdf72efa2560012560606d42a7
:020000040000fa
:2091a000d9e77d49fdf726fa7c49061cfdf722fa011c051c301cfdf7c9fe7849eae7784b84
:020000040000fa
:2091c0009f4200d98be0029776490298fdf77efdfc218905fdf70efafef77ef80500fef7fd
:020000040000fa
:2091e0009bf86b490490fdf771fd011c0298fdf7adfe684902900498fdf768fd0390011cf4
:020000040000fa
:209200000298fdf7a3fe1f2d07dc674a691e8900664b8a583340934206d1ff22c30dff1578
:020000040000fa
:209220001340fb1a082b01dc206025e05a490498fdf74cfd011c03900298fdf787fe011cd5
:020000040000fa
:20924000061c0298fdf782fe0399fdf77ffe534902900498fdf73afd0299fdf777fe039045
:020000040000fa
:20926000011c301cfdf772feff22c30d1340fb1a192b15dc2060029626680298311cfdf712
:020000040000fa
:2092800065fe0399fdf762fe059b6060002b00db61e780231b06f618c018266060607ee778
:020000040000fa
:2092a00043490498fdf712fd071c011c301cfdf74dfe0290011c301cfdf748fe391cfdf73a
:020000040000fa
:2092c00045fe3c49061c0498fdf700fd311cfdf73dfe0390011c0298fdf738fea4e7ff237a
:020000040000fa
:2092e000db059f4205d3011cfdf730fe6060206013e7fe15863ef5057d1b281cfdf7ecffd0
:020000040000fa
:20930000fef70af8011c0790281cfdf71ffe8721c905fdf7dbfc071cfdf7defffdf7fcff29
:020000040000fa
:20932000011c0890051c381cfdf710fe8721c905fdf7ccfc00210990fdf714f803230028c7
:020000040000fa
:2093400006d00021281cfdf70df8434243410133194a21000192022207a80092320000f0fe
:020000040000fa
:209360002df8059b0500002b00dbf4e68022236812069b18236063689b1863600fe7c0468b
:020000040000fa
:20938000d80f493fe3cb1640f0ffff7fd00fc93f800fc93f434435370044353708a3852e6e
:020000040000fa
:2093a000800f494384f9223fc8a9000000ffff7f00a3852e32318d2448aa0000f0b5ddb038
:020000040000fa
:2093c0000692629a0793c84b9200d35809900493079b0291013b059300230193069b0433c7
:020000040000fa
:2093e00007db0721069bda1ed3170b409b18db100193019b20ae0133db000893089a069b0c
:020000040000fa
:209400009b1a0093059a019b9d1a2c00049b9f18631b9f420dda079c48af079b049ae31a73
:020000040000fa
:209420009a4225dba30020aa9e1800230025039316e00020002c04db639aa300d058fdf772
:020000040000fa
:209440006bff01c60134e3e7099aab003168d058fdf73cfc011c0398fdf7ccf80135039068
:020000040000fa
:20946000059b043e9d42efdd039b013408c7d4e7049b0caa9b009b180b93019b639a9b008d
:020000040000fa
:20948000d318049f0a93f0210cae34003d000caabb005218d3580193002d64dc009901982c
:020000040000fa
:2094a00000f02afaf8218905041cfdf70ffc00f079fa8221c905fdf709fc011c201cfdf7b8
:020000040000fa
:2094c00045fd041cfdf708ff0390fdf725ff011c201cfdf73bfd009b041c002b63dd0820b1
:020000040000fa
:2094e0007b1e9b000caa9a580099039d401a110001416d188140521a0ca95a5007230099d6
:020000040000fa
:2095000003955b1a1a410192019b002b5cdd039b00220133039380235b0015000121ff2072
:020000040000fa
:209520009c46974200dd82e0009b002b05dd012b00d18be0022b00d191e0019b022b43d1d5
:020000040000fa
:20954000fe20211c8005fdf701fd041c002d3bd0fe200099800500f0cff9011c201cfdf7a0
:020000040000fa
:20956000f5fc041c30e0ee2101988905fdf7aefbfdf7b2fefdf7d0fe8721c9050390fdf794
:020000040000fa
:20958000a5fb011c0198fdf7e1fcfdf7a5fef021013d0caaab00521801c4d1580398fdf776
:020000040000fa
:2095a00029f8019078e7009b002b06d17b1e9b000caa9b58db110193a6e7fc218905fcf775
:020000040000fa
:2095c000f5fe002830d101900021201cfcf7cafe002800d18ce000227b1e04998b4244da1e
:020000040000fa
:2095e000002a5cd0009b013f083b00930caabb009b58002bf6d0fe200099800500f07cf96e
:020000040000fa
:209600003d00041c002d00dba8e03c00374b0693002c00dacfe0a30048aa9b1805933b1b1b
:020000040000fa
:20962000002600250093bae0022301936fe73368002d09d1002b03d06546eb1a33600b00b5
:020000040000fa
:209640001d00013204366ce7c31af7e77f217b1e9b000caa9a580a400ca95a506de77b1e60
:020000040000fa
:209660009b000caa3f219a58f5e799000ca80958013b0a43b1e701330b999a0052428a58b4
:020000040000fa
:20968000002af8d0079a20a9ba189200fb187e1c8c180193019bb34203da1f00f3e601239b
:020000040000fa
:2096a000eae7b30003930a9bb2009858fdf734fe002700252060059b9f4207ddf021039a44
:020000040000fa
:2096c0000cab5b189d5001360434e3e7bb0009995a42c958a058fdf7f9fa011c281cfcf7ed
:020000040000fa
:2096e00089ff0137051ce6e760ad00006cad0000089b069a201c991a00f0fef88721c90508
:020000040000fa
:20970000041cfcf753fe002821d0ee21201c8905fdf7dcfafdf7e0fdfdf7fefd8721c905f3
:020000040000fa
:20972000051cfdf7d3fa011c201cfdf70ffcfdf7d3fdbe000cab9851009b281c0833009320
:020000040000fa
:20974000fdf7cafd0137bc000cab185153e7201cfdf7c2fdbd000cab58514ce70cabae005c
:020000040000fa
:20976000f058fdf7d9fd211cfdf7b0faf022ee210cab9b1898518905201cfdf7a7fa013deb
:020000040000fa
:20978000041c3fe7059aab00d158069a01359858fdf79cfa011c301cfcf72cff061c049b78
:020000040000fa
:2097a0009d4202dc009b9d42ecdd009b013c9a0034abd6502ce7629b022b08dc002b58dcb2
:020000040000fa
:2097c00033d00720039b034018005db0f0bd629b032bf6d1bb0034aad61834003d00043c82
:020000040000fa
:2097e000002d50dc3d00043e012d61dc002034ac012f71dc0199349a6368002972d102996f
:020000040000fa
:209800004b600b000a609860dbe7bb001959fcf7f1fe013f002ff8da019b002b02d08023e2
:020000040000fa
:209820001b06c018029b1860cbe7002034acf1e7a3005959fcf7defe013c002cf8da019a96
:020000040000fa
:20984000031c002a02d080231b06c318029a011c13603498fdf77afb012434ada7420cda18
:020000040000fa
:20986000019b002b02d080231b06c018029b5860a7e73c00002034addfe7a3005959fcf785
:020000040000fa
:20988000b9fe0134eae72368013d009363680098191c0493fcf7aefe011c05900098fdf7a3
:020000040000fa
:2098a00055fb0499fcf7a6fe059b6060236096e73368013d009373680098191c0493fcf726
:020000040000fa
:2098c00099fe011c041c0098fdf740fb0499fcf791fe3460706086e7bb00e158fcf78afe8e
:020000040000fa
:2098e000013f85e78021029c09065b185218636022602300401886e7430010b502000c004e
:020000040000fa
:2099000059081b0e14d1002917d09821c905fdf7ddf91849c315dbb20200193bc00f8c42be
:020000040000fa
:209920001adb15498c4209ddd00f00f031f804e0ff2bf6d1011cfcf75dfe10bde318fe2bf7
:020000040000fa
:20994000f2dc002b04dd0d48db0510401843f4e71900183103dad00f00f012f8ede7cc2199
:020000040000fa
:209960001933d805054b89051a401043fdf7aef9e3e7c046b03cffff50c30000ffff7f80ce
:020000040000fa
:20998000002802d08020000670470020fce70000002801d002487047ff20c005fbe7c046a7
:020000040000fa
:2099a000000080ff42005108120e7f3a10b50400162a1cdc0300002a0dda0023984208dac0
:020000040000fa
:2099c0004b1e9941fe224b4292051340802212069b18181c12e00a49114108420ed0002825
:020000040000fa
:2099e00003da80200004104123188b43f1e7ff23db05994202d3011cfcf7fcfd10bdc04626
:020000040000fa
:209a0000ffff7f00d0400b00d1409c46203ad340184352426346934018437047d0400b00b6
:020000040000fa
:209a20001141203a03d49c461341184363465242934018437047c0469140030090409c4664
:020000040000fa
:209a4000203a9340194352426346d340194370474561737954696d65722d763200616c7471
:020000040000fa
:209a600075736d657472756d2e6f726700312e392e313700006d616e756661637475726525
:020000040000fa
:209a800072202020202025730a70726f647563742020202020202020202025730a736572e5
:020000040000fa
:209aa00069616c2d6e756d6265722020202025750a63757272656e742d666c6967687420c8
:020000040000fa
:209ac000202025750a6c6f672d666f726d61742020202020202025750a6c6f672d73706173
:020000040000fa
:209ae00063650920256c750a70726f6772616d2d73706163652020202025750a616c746966
:020000040000fa
:209b0000747564652d3332202020202020310a00736f6674776172652d76657273696f6e68
:020000040000fa
:209b200020252e38730a0053796e746178206572726f720a0065626f6f7400636d640025b0
:020000040000fa
:209b40002d3230732025730a004265657065722073657474696e673a2025640a00507972a8
:020000040000fa
:209b60006f2074696d653a2025640a004d617820666c69676874206c6f673a202564206b26
:020000040000fa
:209b8000420a00506164206f7269656e746174696f6e3a2025640a00416363656c206361ef
:020000040000fa
:209ba0006c202b31673a202564202d31673a2025640a00494d552063616c20616c6f6e6735
:020000040000fa
:209bc000202564206163726f7373202564207468726f7567682025640a004f7269656e7443
:020000040000fa
:209be00020616e74656e6e6120257320616e642070726573732061206b65792e2e2e000d87
:020000040000fa
:209c00000a0043616c6962726174696e672e2e2e005361766564004e6f7468696e672074f2
:020000040000fa
:209c20006f2073617665004e3043414c4c0053746f72616765206d75737420626520656db5
:020000040000fa
:209c4000707479206265666f7265206368616e67696e67206c6f672073697a6500466c695d
:020000040000fa
:209c6000676874206c6f67206d6178202575206b420a00757000646f776e00496e76616cb1
:020000040000fa
:209c8000696420616363656c3a207570202825642920646f776e20282564290a00436f6eaa
:020000040000fa
:209ca0006669672076657273696f6e3a2025642e25640a002532643a20776368616e202539
:020000040000fa
:209cc00030387820616c61726d202535642025730a0053746f726167652073697a653a20cd
:020000040000fa
:209ce000256c640a0053746f7261676520657261736520756e69743a20256c640a00446f74
:020000040000fa
:209d0000497400444d41202573206374726c202530347820696e7470656e642025303478d3
:020000040000fa
:209d200020696e74737461747573202530346c780a0020627573796368202530346c782022
:020000040000fa
:209d400070656e646368202530346c7820616374697665202530386c782063686374726c37
:020000040000fa
:209d60006120253032780a002063686374726c62202530386c78206368696e74666c6167f6
:020000040000fa
:209d8000202530327820636873746174757320253032780a002062746374726c2025303498
:020000040000fa
:209da00078206274636e7420253034782073726361646472202530386c782064737461640b
:020000040000fa
:209dc0006472202530386c78206465736361646472202530386c780a00424d493038383a75
:020000040000fa
:209de0002025376420253764202537642025376420253764202537640a00626d6930383841
:020000040000fa
:209e0000004d4d43353938333a2025642025642025640a006d6d63353938330044657465b5
:020000040000fa
:209e20006374656420636869707320312073697a6520256c640a007469636b3a2025356c35
:020000040000fa
:209e40007520413a2025356420423a2025356420626174743a202535640a007265706f7285
:020000040000fa
:209e60007400257325730049676e697465723a202564205374617475733a2025730a005099
:020000040000fa
:209e800079726f2d636f756e743a2025640a005079726f202532643a20003c646973616207
:020000040000fa
:209ea0006c65643e0025366c64200020202020202020003c6e3e2000696e76616c696420f5
:020000040000fa
:209ec0007079726f206368616e6e656c20256c750a00696e76616c6964207079726f206638
:020000040000fa
:209ee00069656c642025730a00616f5f7079726f5f6d616e75616c2025640a007079726faf
:020000040000fa
:209f000000616363656c206c65737320286d2f7373202a2031362900616363656c206772bd
:020000040000fa
:209f2000656174657220286d2f7373202a20313629007370656564206c65737320286d2f80
:020000040000fa
:209f400073202a20313629007370656564206772656174657220286d2f73202a2031362928
:020000040000fa
:209f600000686569676874206c65737320286d290068656967687420677265617465722010
:020000040000fa
:209f8000286d29006f7269656e74206c657373202864656729006f7269656e74206772650b
:020000040000fa
:209fa000617465722028646567290074696d65206c657373202873202a203130302900747b
:020000040000fa
:209fc000696d652067726561746572202873202a2031303029007374617465206c65737365
:020000040000fa
:209fe0000073746174652067726561746572206f7220657175616c00617363656e64696eb8
:020000040000fa
:20a00000670064657363656e64696e67006166746572206d6f746f720064656c61792062d1
:020000040000fa
:20a0200065666f726520666972696e67202873202a203130302900666c6967687400756e30
:020000040000fa
:20a040006b6e6f776e00726561647900616374697665006f70656e004e6f207375636820e0
:020000040000fa
:20a06000666c696768743a20256c640a00457261736564004661696c656420746f20657276
:020000040000fa
:20a0800061736500666c6967687420256c6420737461727420257820656e642025780a00cb
:020000040000fa
:20a0a000736c6f742025642020737461727420257820656e642025780a00646f6e65006cda
:020000040000fa
:20a0c0006f6700696e66006e616e00286e756c6c29000000082008003b13000010a10000f5
:020000040000fa
:20a0e0005d21000017a10000631600001fa100001917000034a10000af12000043a1000047
:020000040000fa
:20a10000a11200004da1000000000000000000003f0048656c700054005461736b73004537
:020000040000fa
:20a12000203c30206f66662c2031206f6e3e004563686f00722065626f6f74005265626fce
:020000040000fa
:20a140006f7400760056657273696f6e00580053776974636820746f20626f6f74206c6f24
:020000040000fa
:20a16000616465720000000023a20000511c00006118000048a20000111c00004918000020
:020000040000fa
:20a1800079a20000a91b00002d18000097a20000f55400004d540000ada20000811b00008d
:020000040000fa
:20a1a00015180000c8a20000591b0000fd170000f9a200007d1d00000000000000a30000a8
:020000040000fa
:20a1c000b11900000000000012a30000c91700000000000000000000000000000000000020
:020000040000fa
:20a1e00069190000f0a10000000000000000000063203c7661723e203c76616c75653e004f
:020000040000fa
:20a2000053657420636f6e66696720283f20666f722068656c702c207320746f2073686f99
:020000040000fa
:20a2200077290061203c2b673e203c2d673e00416363656c2063616c696220283020666f63
:020000040000fa
:20a2400072206175746f29006f203c3020616e74656e6e612075702c203120616e74656ed2
:020000040000fa
:20a260006e6120646f776e3e00506164206f7269656e746174696f6e006c203c73697a6595
:020000040000fa
:20a280003e00466c69676874206c6f672073697a6520286b42290050203c6e2c3f3e0050b4
:020000040000fa
:20a2a00079726f206368616e6e656c730049203c7469636b733e005079726f206669726963
:020000040000fa
:20a2c0006e672074696d650062203c76616c3e0042656570657220746f6e652028667265ed
:020000040000fa
:20a2e00071203d20312f322028323465362f333229202f206265657000730053686f7700b9
:020000040000fa
:20a300007700577269746520746f20656570726f6d003f0048656c70000000000c0000201c
:020000040000fa
:20a320005d22000048a30000e922000057a30000a52400006ca300008124000084a300000a
:020000040000fa
:20a340000000000000000000660053686f772073746f726167650065203c626c6f636b3ed7
:020000040000fa
:20a360000044756d7020666c617368007a203c626c6f636b3e004572617365203c626c6f71
:020000040000fa
:20a38000636b3e005a203c6b65793e00457261736520616c6c2e203c6b65793e20697320fe
:020000040000fa
:20a3a000646f697420776974682044264900000000080042000c00420010004200140042fe
:020000040000fa
:20a3c00000180042001c0042052f0000d8a300000000000000000000490053686f772042ca
:020000040000fa
:20a3e0004d4930383820737461747573000000008132000000a4000000000000000000000c
:020000040000fa
:20a400004d0053686f77204d4d43353938332073746174757300000000020a182d3900002a
:020000040000fa
:20a420002ca4000000000000000000006100446973706c61792063757272656e742041444d
:020000040000fa
:20a44000432076616c756573000302340c242c0b1a144c00010002100200041004000610ac
:020000040000fa
:20a460000800081010000a1020000c1040000e1080001010000112100002141000201610c9
:020000040000fa
:20a48000004018080080190800101a10613c000001000200019f0000613e0000020004009c
:020000040000fa
:20a4a000189f0000733c000004000600329f0000733e000008000800489f0000683c00000f
:020000040000fa
:20a4c00010000a00619f0000683e000020000c00719f00006f3c000040000e00849f000064
:020000040000fa
:20a4e0006f3e000080001000969f0000743c000000011400ab9f0000743e0000000218000f
:020000040000fa
:20a50000bf9f0000663c000000402000d69f0000663e3d0000802100e19f00004100000023
:020000040000fa
:20a520000004ff00f89f0000440000000008ff0002a000006d000000001022000da0000048
:020000040000fa
:20a540006400000000201c0019a00000000000000000ff0000000000315a000070a5000003
:020000040000fa
:20a56000295a0000aba50000000000000000000069203c6b65793e207b6d61696e7c64722a
:020000040000fa
:20a580006f6775657d00466972652069676e697465722e203c6b65793e20697320646f698d
:020000040000fa
:20a5a00074207769746820442649007400546573742069676e697465720000003ea0000074
:020000040000fa
:20a5c00046a000004ca0000053a00000695c0000e4a50000995b0000f0a5000000000000df
:020000040000fa
:20a5e000000000006c004c697374206c6f67730064203c666c696768742d6e756d6265728a
:020000040000fa
:20a600003e0044656c65746520666c6967687400e86a0000ce690000f86900005e6a000059
:020000040000fa
:20a62000f8690000926a0000f86900005e6a0000ce690000ce690000926a00005e6a000062
:020000040000fa
:20a64000e4690000e4690000e46900009c6a0000ce690000ce690000f8690000206b0000b3
:020000040000fa
:20a66000f8690000926a0000f8690000206b0000ce690000ce690000926a0000206b00009c
:020000040000fa
:20a68000e4690000e4690000e46900000000000000000000000000000000000000000000d3
:020000040000fa
:20a6a0000000004095596959555554551555555604051541105455404551554440455044a2
:020000040000fa
:20a6c000505555450040004040044496655556554540455451411540559155555555405168
:020000040000fa
:20a6e00005010000544554544555050400100410140440000000014055551541540400005b
:020000040000fa
:20a70000440001000000004041000044504445505400555554556551004000400100000127
:020000040000fa
:20a72000000501001154515154555505000000000000000000000000010000000000000008
:020000040000fa
:20a74000050000000000000019000000000000007d000000000000007102000000000000eb
:020000040000fa
:20a76000350c000000000000093d0000000000002d31010000000000e1f505000000000018
:020000040000fa
:20a7800065cd1d0000000000f902950000000000dd0ee90200000000514a8d0e00000000ce
:020000040000fa
:20a7a0009573c24800000000e941cc6b010000008d49fd1a07000000c16ff2862300000066
:020000040000fa
:20a7c000c52ebca2b1000000d9e9ac2d780300003d9160e45811000031d6e275bc56000076
:020000040000fa
:20a7e000f52e6e4daeb10100c9ea268367780800ed95c28f055a2a00a1edccce1bc2d300a4
:020000040000fa
:20a8000025a4000a8bca2204000000000000000000000000000000100000000000000000da
:020000040000fa
:20a82000b9340332b7f4ad1410db1ab30892540e0d307d951447ba1a66088f4d26adc66d08
:020000040000fa
:20a84000f598bf85e2b74511ca96853d92bd1debfca11860dcef52163c92ae220bb8c1b4a1
:020000040000fa
:20a86000839d2d5b0562da1c304c7e8f4e8bb25b16f4529f8b56a512fbd4827643ed8af060
:020000040000fa
:20a880008fe7f9311565191850f19bd94a13eeb4284cf0a686c1251f035fc270cb9e4916c8
:020000040000fa
:20a8a000e642889c44eb2014b0650836ad6ea58585f0ca14e2fd031a0b899979d5b13d0990
:020000040000fa
:20a8c000d8da973a35ebcf10ac363f5e73bb38cf3e6752fa44afba1501000000000000008e
:020000040000fa
:20a8e0000000000000000020345065c05fc9a652bb13cbaec440c21806c8df7100d5a87c33
:020000040000fa
:20a90000f56f0fda58fc27136e4756357d24206502c7e768e48ca41de9e60268d7cd396136
:020000040000fa
:20a920007977fcc2405bef16798cde43ffa751f991f3b278f5bdbe11e857e9d6e8bee87b7d
:020000040000fa
:20a94000b054ac8f848d751bea23a499e9f9d38bb7a3714061da3e15cee33ecb73f948087e
:020000040000fa
:20a960008c97b427d51b7010a2bfefb9eb8532154db44db49bbb6f1996b6076cf8e7eead90
:020000040000fa
:20a9800036d9b4f59135ae13222218af4e6a684d91daaa3d4f40741e9fbd9ee006a1c098b4
:020000040000fa
:20a9a00057c2a7fda40e90170e7d497173e3208fb220d87605143b12853d7434811343b0c0
:020000040000fa
:20a9c000ad297a5f27f4351c000fc93f000f494000cb9640000fc9400053fb4000cb164144
:020000040000fa
:20a9e00000ed2f41000f49410031624100537b41003a8a4100cb9641005ca34100edaf41ba
:020000040000fa
:20aa0000007ebc41000fc94100a0d5410031e24100c2ee410053fb4100f20342003a0a425b
:020000040000fa
:20aa20000083104200cb164200141d42005c234200a5294200ed2f4200363642007e3c42d2
:020000040000fa
:20aa400000c74242000f4942a2000000f9000000830000006e0000004e00000044000000f3
:020000040000fa
:20aa60001500000029000000fc0000002700000057000000d1000000f50000003400000024
:020000040000fa
:20aa8000dd000000c0000000db0000006200000095000000990000003c000000430000002f
:020000040000fa
:20aaa0009000000041000000fe0000005100000063000000ab000000de000000bb000000cf
:020000040000fa
:20aac000c500000061000000b7000000240000006e0000003a000000420000004d0000003e
:020000040000fa
:20aae000d2000000e000000006000000490000002e000000ea00000009000000d100000063
:020000040000fa
:20ab0000920000001c000000fe0000001d000000eb0000001c000000b1000000290000008b
:020000040000fa
:20ab2000a70000003e000000e80000008200000035000000f50000002e000000bb000000b3
:020000040000fa
:20ab40004400000084000000e90000009c0000007000000026000000b40000005f000000ff
:020000040000fa
:20ab60007e000000410000003900000091000000d600000039000000830000005300000067
:020000040000fa
:20ab800039000000f40000009c000000840000005f0000008b000000bd000000f9000000c8
:020000040000fa
:20aba000280000003b0000001f000000f800000097000000ff000000de00000005000000a2
:020000040000fa
:20abc000980000000f000000ef0000002f000000110000008b0000005a0000000a000000b0
:020000040000fa
:20abe0006d0000001f0000006d000000360000007e000000cf00000027000000cb000000e7
:020000040000fa
:20ac000009000000b70000004f000000460000003f000000660000009e0000005f0000003d
:020000040000fa
:20ac2000ea0000002d0000007500000027000000ba000000c7000000eb000000e500000010
:020000040000fa
:20ac4000f10000007b0000003d0000000700000039000000f70000008a0000005200000038
:020000040000fa
:20ac600092000000ea0000006b000000fb0000005f000000b10000001f0000008d00000036
:020000040000fa
:20ac80005d0000000800000056000000030000003000000046000000fc0000007b00000009
:020000040000fa
:20aca0006b000000ab000000f0000000cf000000bc000000200000009a000000f400000055
:020000040000fa
:20acc000360000001d000000a9000000e300000091000000610000005e000000e60000005f
:020000040000fa
:20ace0001b000000080000006500000099000000850000005f00000014000000a00000009b
:020000040000fa
:20ad000068000000400000008d000000ff000000d8000000800000004d00000073000000e7
:020000040000fa
:20ad2000270000003100000006000000060000001500000056000000ca0000007300000007
:020000040000fa
:20ad4000a8000000c900000060000000e20000007b000000c00000008c0000006b0000000e
:020000040000fa
:20ad60000400000007000000090000000000c93f0000f0390000da370000a2330000842ef6
:020000040000fa
:20ad80000000502b0000c2270000d0220000c41f0000c61b0000441700000300ed2100002d
:020000040000fa
:14ada00035220000092200000100000000c201000000080051
:00000001ff
